:0200000480007A
:10000000B72F0000938F0F8073900F306F00400365
:100010001300000013000000130000001300000094
:100020001300000013000000130000001300000084
:100030001300000013000000130000001300000074
:100040009702000093824211739052309300000097
:10005000130100009301000013020000930200004E
:100060001303000093030000130400009304000036
:10007000130500009305000013060000930600001E
:100080001307000093070000130800009308000006
:100090001309000093090000130A0000930A0000EE
:1000A000130B0000930B0000130C0000930C0000D6
:1000B000130D0000930D0000130E0000930E0000BE
:1000C000130F0000930F000097110200938141CCA1
:1000D000170502001305054F97A503009385858139
:1000E00013060000EF00001A170502001305C549AA
:1000F000970502009385854913060000EF008018DC
:1001000017A503001305457F97B503009385857EEA
:1001100037B6ABAB1306B6BAEF00C01617B1030083
:100120001301817DEF70802A9392120093D2120006
:100130009382D2FF638A02008322010013014100EF
:100140006F0000177300203083220100130141006B
:10015000730020301301C1FF23205100F32220340B
:10016000E3C402FC8322010013014100130141F8A2
:1001700023221100232421002326310023284100BB
:10018000232A5100232C6100232E71002320810299
:10019000232291022324A1022326B1022328C10293
:1001A000232AD102232CE102232EF1022320010570
:1001B0002322110523242105232631052328410567
:1001C000232A5105232C6105232E71052320810745
:1001D000232291072324A1072326B1072328C1073F
:1001E000232AD107232CE107232EF107732520347E
:1001F000F3251034130601006F000000731015344E
:1002000083204100032181008321C10003220101D9
:1002100083224101032381018323C10103240102BD
:1002200083244102032581028325C10203260103A1
:1002300083264103032781038327C1030328010485
:1002400083284104032981048329C104032A010569
:10025000832A4105032B8105832BC105032C01064D
:10026000832C4106032D8106832DC106032E010731
:10027000832E4107032F8107832FC1071301C10775
:10028000730020302320C5006376B50013054500B8
:100290006FF05FFF678000000000000000000000BA
:1002A000000000000000000000000000000000004E
:1002B000130101F8232011002322210023243100FF
:1002C0002326410023285100232A6100232C71009A
:1002D000232E8100232091022322A1022324B10294
:1002E0002326C1022328D102232AE102232CF10272
:1002F000232E010323201105232221052324310568
:100300002326410523285105232A6105232C710545
:10031000232E8105232091072322A1072324B1073F
:100320002326C1072328D107232AE107232CF1071D
:100330009702020083A2422523A02200F322103458
:10034000232E5106EF00404E170102000321C12366
:10035000032101008322C10773901234B7220000E9
:100360009382028873A00230832001000322C1001F
:100370008322010103234101832381010324C1015D
:100380008324010203254102832581020326C10241
:100390008326010303274103832781030328C10325
:1003A000832801040329410483298104032AC10409
:1003B000832A0105032B4105832B8105032CC105ED
:1003C000832C0106032D4106832D8106032EC106D1
:1003D000832E0107032F4107832F81071301010893
:1003E00073002030970202009382C21D23A01200E6
:1003F00023A2220023A4320023A6420023A85200F5
:1004000023AA620023AC720023AE820023A09202D2
:1004100023A2A20223A4B20223A6C20223A8D202CC
:1004200023AAE20223ACF20223AE020323A01205A8
:1004300023A2220523A4320523A6420523A85205A0
:1004400023AA620523AC720523AE820523A092077E
:1004500023A2A20723A4B20723A6C20723A8D20778
:1004600023AAE20723ACF207EF00402B170102009A
:1004700003218111032101008322C10773901234EB
:10048000B72200009382028873A00230832001000B
:100490000322C1008322010103234101832381013F
:1004A0000324C10183240102032541028325810223
:1004B0000326C10283260103032741038327810307
:1004C0000328C103832801040329410483298104EB
:1004D000032AC104832A0105032B4105832B8105CF
:1004E000032CC105832C0106032D4106832D8106B3
:1004F000032EC106832E0107032F4107832F810797
:100500001301010873002030970202009382820BCE
:1005100083A0020003A1420083A1820003A2C200C3
:1005200083A2020103A3420183A3820103A4C201A7
:1005300083A4020203A5420283A5820203A6C2028B
:1005400083A6020303A7420383A7820303A8C2036F
:1005500083A8020403A9420483A9820403AAC20453
:1005600083AA020503AB420583AB820503ACC20537
:1005700083AC020603AD420683AD820603AEC2061B
:1005800083AE020703AFC20983AF82076780000012
:1005900073700430130101F823201100232221007D
:1005A000232431002326410023285100232A6100FF
:1005B000232C7100232E8100232091022322A102EB
:1005C0002324B1022326C1022328D102232AE102D7
:1005D000232CF102232E01032320110523222105C0
:1005E000232431052326410523285105232A6105AB
:1005F000232C7105232E8105232091072322A10797
:100600002324B1072326C1072328D107232AE10782
:10061000232CF1079702020083A202F723A02200F5
:10062000232E1106EF20505E170102000321C1F5B1
:10063000032101008322C10773901234B722000006
:100640009382028873A00230832001000322C1003C
:100650008322010103234101832381010324C1017A
:100660008324010203254102832581020326C1025E
:100670008326010303274103832781030328C10342
:10068000832801040329410483298104032AC10426
:10069000832A0105032B4105832B8105032CC1050A
:1006A000832C0106032D4106832D8106032EC106EE
:1006B000832E0107032F4107832F810713010108B0
:1006C00073002030970702009387C7EC83A70700C9
:1006D00003A8470083A70700170702001307C7EB0B
:1006E000032507009305803E13060000B386B7007C
:1006F00093880600B3B8F8003307C800B387E80052
:100700001387070093870600130807002320F500CE
:10071000232205011300000067800000130101FF80
:1007200023261100EFF01FFA9307000873A047304B
:10073000130000008320C100130101016780000045
:10074000970702009387C7E403A707009307F0FF0A
:100750006306F700737004306F000000737004309C
:100760006F000000130101FF2326A1008327C100B1
:1007700073904730130000001301010167800000EF
:10078000130101FFF32740302326F10073F04330BB
:100790008327C10013850700130101016780000052
:1007A000130101FF2326A1002324B1002322C1004D
:1007B0008327C1009387C7FF2326F1000327810009
:1007C0008327C10023A0E7008327C100938787FA0E
:1007D0002326F100032741008327C10023A0E7005F
:1007E0008327C100938787FE2326F10093870100AA
:1007F000138707008327C10023A0E7008327C100D8
:10080000938747FF2326F10017070000130787F39C
:100810008327C10023A0E7008327C10013850700B9
:100820001301010167800000130101FF232611005D
:10083000EFF05FE9EF20D013930705006384070012
:10084000EF20903C130000008320C1001301010140
:1008500067800000130101FF2326A1008327C10048
:10086000138787008327C10023A2E7008327C100E5
:100870001307F0FF23A4E7008327C1001387870035
:100880008327C10023A6E7008327C10013878700C1
:100890008327C10023A8E7008327C10023A0070006
:1008A000130000001301010167800000130101FF24
:1008B0002326A1008327C10023A8070013000000FE
:1008C0001301010167800000130101FE2326A1002E
:1008D0002324B1008327C10083A74700232EF10002
:1008E000832781000327C10123A2E7008327C101D9
:1008F00003A787008327810023A4E7008327C10182
:1009000083A787000327810023A2E7008327C10173
:100910000327810023A4E700832781000327C10068
:1009200023A8E7008327C10083A7070013871700C8
:100930008327C10023A0E700130000001301010278
:1009400067800000130101FE2326A1002324B100CB
:100950008327810083A70700232CF100032781014F
:100960009307F0FF631AF7008327C10083A70701ED
:10097000232EF1006F0040038327C1009387870077
:10098000232EF1006F0000018327C10183A74700D8
:10099000232EF1008327C10183A7470083A7070007
:1009A00003278101E372F7FE8327C10103A74700F4
:1009B0008327810023A2E7008327810083A74700C4
:1009C0000327810023A4E700832781000327C101B7
:1009D00023A4E7008327C1010327810023A2E700A6
:1009E000832781000327C10023A8E7008327C100D4
:1009F00083A70700138717008327C10023A0E70000
:100A0000130000001301010267800000130101FEC2
:100A10002326A1008327C10083A70701232EF1000D
:100A20008327C10083A747000327C100032787004E
:100A300023A4E7008327C10083A787000327C10001
:100A40000327470023A2E7008327C10183A74700AC
:100A50000327C100631AF7008327C10003A787009B
:100A60008327C10123A2E7008327C10023A8070031
:100A70008327C10183A707001387F7FF8327C101DD
:100A800023A0E7008327C10183A707001385070080
:100A90001301010267800000130101FD23261102EA
:100AA0002326A1002324B1008327C100232EF100B7
:100AB0008327C10163960700737004306F00000044
:100AC000EF30103F8327C10103A707008327C1012F
:100AD00083A6C7038327C10183A70704B387F60250
:100AE0003307F7008327C10123A2E7008327C10151
:100AF00023AC07028327C10103A707008327C10195
:100B000023A4E7008327C10103A707008327C101AE
:100B100083A7C7039386F7FF8327C10183A7070431
:100B2000B387F6023307F7008327C10123A6E70046
:100B30008327C1011307F0FF23A2E7048327C10124
:100B40001307F0FF23A4E70483278100639A0702B9
:100B50008327C10183A70701638407048327C10199
:100B60009387070113850700EF20D04B130705007B
:100B7000930710006316F702EFF09FA16F00400289
:100B80008327C1019387070113850700EFF09FCCEE
:100B90008327C1019387470213850700EFF09FCB9E
:100BA000EF30103593071000138507008320C10232
:100BB0001301010367800000130101FD23261102C8
:100BC0002326A1002324B10093070600A303F1000C
:100BD000232C01008327C100639607007370043043
:100BE0006F0000008327810063960700232E010019
:100BF0006F0080010327C10083278100B307F7023C
:100C000093871700232EF1008327C101938747059F
:100C100013850700EF50006E232AA10083274101AE
:100C20006382070683278100639A070083274101B7
:100C30000327410123A0E7006F0040018327410102
:100C4000138747058327410123A0E700832741013C
:100C50000327C10023AEE702832741010327810058
:100C600023A0E7049305100003254101EFF0DFE224
:100C700083274101034771002388E704832741014B
:100C8000232CF100832781016396070073700430E1
:100C90006F00000083278101138507008320C102B4
:100CA0001301010367800000130101FD23261102D7
:100CB00093070500A307F10013054005EF5080637B
:100CC000232EA1008327C101638C07088327C1015C
:100CD00023A207008327C10123A007008327C101A6
:100CE00023A407008327C10123A607008327C1018E
:100CF00023AC07028327C1011307100023AEE702CC
:100D00008327C10123A007048327C1011307F0FF34
:100D100023A2E7048327C1011307F0FF23A4E704FC
:100D20008327C1010347F1002388E7048327C1011A
:100D30009387070113850700EFF0DFB18327C10117
:100D40009387470213850700EFF0DFB0930600009A
:100D500013060000930500000325C101EF00001EEB
:100D60008327C101138507008320C10213010103FA
:100D700067800000130101FD232611022324810254
:100D80002326A1008327C100232CF10083278101A2
:100D900063960700737004306F00000083278101A1
:100DA00003A44700EF300060930705006312F404CA
:100DB0008327810183A7C7001387F7FF832781015A
:100DC00023A6E7008327810183A7C700639C070050
:100DD000930600001306000093050000032581011F
:100DE000EF00C01593071000232EF1006F00800064
:100DF000232E01008327C101138507008320C10230
:100E0000032481021301010367800000130101FD27
:100E100023261102232481022326A1002324B100CA
:100E20008327C100232CF1008327810163960700EB
:100E3000737004306F0000008327810103A4470012
:100E4000EF304056930705006312F40283278101B7
:100E500083A7C700138717008327810123A6E70014
:100E600093071000232EF1006F00C00393060000CB
:100E7000032681009305000003258101EF00C0587F
:100E8000232EA1000327C10193071000631CF70064
:100E90008327810183A7C700138717008327810158
:100EA00023A6E7008327C101138507008320C10221
:100EB000032481021301010367800000130101FD77
:100EC000232611022326A1002324B1008327C10079
:100ED00063960700737004306F00000003278100E1
:100EE0008327C10063F6E700737004306F000000D1
:100EF00013062000930500000325C100EFF0DFCBAF
:100F0000232EA1008327C101638807008327C10125
:100F10000327810023ACE7028327C1016396070002
:100F2000737004306F0000008327C1011385070030
:100F30008320C1021301010367800000130101FC3B
:100F4000232E11022326A1002324B1002322C10055
:100F50002320D100232601028327C1002324F1028C
:100F60008327810263960700737004306F000000CE
:100F700083278100639807008327810283A70704E2
:100F800063960700930710006F008000930700002E
:100F900063960700737004306F00000003270100A0
:100FA00093072000631AF7008327810203A7C70372
:100FB000930710006316F700930710006F0080007E
:100FC0009307000063960700737004306F00000001
:100FD000EF30803F930705006396070083274100A9
:100FE00063960700930710006F00800093070000CE
:100FF00063960700737004306F000000EF30406BA1
:101000008327810203A787038327810283A7C7035E
:101010006368F70003270100930720006310F706B9
:10102000032601008325810003258102EF00101CA7
:101030002322A1028327810283A747026384070238
:10104000832781029387470213850700EF20807D65
:101050001307050093071000631CF700EFF04FD350
:101060006F0000018327410263840700EFF04FD235
:10107000EF300068930710006F00400F8327410096
:1010800063980700EF30C066930700006F00000E02
:101090008327C102639C07009307C10113850700E2
:1010A000EF20501D930710002326F102EF3040641B
:1010B000EF10D049EF30C05F8327810203A74704B8
:1010C0009307F0FF6316F7008327810223A207042A
:1010D0008327810203A787049307F0FF6316F700B5
:1010E0008327810223A40704EF30806013074100A7
:1010F0009307C1019305070013850700EF20501CDB
:1011000093070500639C070403258102EF00504606
:1011100093070500638C07028327810293870701E9
:10112000032741009305070013850700EF20004ABD
:1011300003258102EF00902CEF10904393070500E8
:10114000E39E07EAEFF0CFC46FF05FEB0325810267
:10115000EF00D02AEF10D0416FF05FEA0325810243
:10116000EF00D029EF10D04093070000138507004F
:101170008320C1031301010467800000130101FDF6
:10118000232611022326A1002324B1002322C1001B
:101190002320D1008327C100232CF1008327810164
:1011A00063960700737004306F000000832781008E
:1011B000639807008327810183A7070463960700CC
:1011C000930710006F0080009307000063960700EC
:1011D000737004306F0000000327010093072000A4
:1011E000631AF7008327810103A7C7039307100041
:1011F0006316F700930710006F008000930700004C
:1012000063960700737004306F000000EFF04FD753
:1012100093070500232AF1008327810103A7870391
:101220008327810183A7C7036368F70003270100B1
:10123000930720006310F70803260100832581002F
:1012400003258101EF00807A8327810103A78704AA
:101250009307F0FF6310F7048327810183A74702F8
:10126000638407048327810193874702138507005E
:10127000EF20405B93070500638807028327410046
:1012800063840702832741001307100023A0E700AF
:101290006F0080018327810183A7870413871700CC
:1012A0008327810123A4E70493071000232EF10074
:1012B0006F008000232E0100832741011385070062
:1012C000EFF04FCA8327C101138507008320C102B5
:1012D0001301010367800000130101FD23261102A1
:1012E0002326A1002324B1008327C100232CF10071
:1012F0008327810163960700737004306F0000003C
:101300008327810183A70704638607007370043075
:101310006F0000008327810183A7070063980700FF
:101320008327810183A74700639607009307100076
:101330006F0080009307000063960700737004300D
:101340006F000000EFF0CFC393070500232AF100E0
:101350008327810103A787038327810183A7C7030D
:101360006372F7088327810183A787031387170018
:101370008327810123ACE7028327810103A7870428
:101380009307F0FF6310F7048327810183A74702C7
:10139000638407048327810193874702138507002D
:1013A000EF204048930705006388070283278100E8
:1013B00063840702832781001307100023A0E7003E
:1013C0006F0080018327810183A78704138717009B
:1013D0008327810123A4E70493071000232EF10043
:1013E0006F008000232E0100832741011385070031
:1013F000EFF04FB78327C101138507008320C10297
:101400001301010367800000130101FC232E110268
:101410002326A1002324B1002322C1002320D100D0
:10142000232601028327C1002324F102832781029E
:1014300063960700737004306F00000083278100FB
:10144000639807008327810283A707046396070038
:10145000930710006F008000930700006396070059
:10146000737004306F000000EF20107693070500C2
:1014700063960700832741006396070093071000D7
:101480006F008000930700006396070073700430BC
:101490006F000000EF30C0218327810283A78703FC
:1014A0006382070C8327810283A7C7002322F102EE
:1014B0008325810003258102EF00806B83270100D3
:1014C000639207068327810283A787031387F7FFA9
:1014D0008327810223ACE7028327810283A70700C9
:1014E000639A0700EF30802B1307050083278102E2
:1014F00023A2E7008327810283A70701638E0704E5
:10150000832781029387070113850700EF2080312D
:1015100013070500930710006310F704EFF04F87DF
:101520006F008003832781020327410223A6E7007F
:101530008327810283A747026380070283278102F2
:101540009387470213850700EF20C02D93070500FE
:1015500063840700EFF0CF83EF308019930710000A
:101560006F0080118327410063980700EF30401817
:10157000930700006F0040108327C102639C07009F
:101580009307C10113850700EF20C04E9307100099
:101590002326F102EF30C015EF10407BEF304011F1
:1015A0008327810203A747049307F0FF6316F70020
:1015B0008327810223A207048327810203A78704CC
:1015C0009307F0FF6316F7008327810223A4070423
:1015D000EF300012130741009307C1019305070084
:1015E00013850700EF20C04D93070500639E070693
:1015F00003258102EF00406F93070500638E070407
:101600008327810283A70700639E0700EF30400A0B
:101610008327810283A7470013850700EF20D05F4F
:10162000EF30000D83278102938747020327410093
:101630009305070013850700EF10507903258102F9
:10164000EF00C05BEF10C07293070500E39407E45E
:10165000EFE01FF46FF01FE403258102EF00005A52
:10166000EF1000716FF01FE303258102EF000059B6
:10167000EF10007093070000138507008320C1035B
:101680001301010467800000130101FD23261102EC
:101690002326A1002324B1002322C1008327C100F7
:1016A000232CF100832781016396070073700430B7
:1016B0006F00000083278100639807008327810162
:1016C00083A7070463960700930710006F0080004C
:1016D0009307000063960700737004306F000000EA
:1016E000EFF00F8A93070500232AF1008327810179
:1016F00083A7870363880708832581000325810169
:10170000EF0000478327810183A787031387F7FF33
:101710008327810123ACE7028327810103A74704C4
:101720009307F0FF6310F7048327810183A7070164
:1017300063840704832781019387070113850700CA
:10174000EF20400E930705006388070283274100BE
:1017500063840702832741001307100023A0E700DA
:101760006F0080018327810183A747041387170037
:101770008327810123A2E70493071000232EF100A1
:101780006F008000232E010083274101138507008D
:10179000EFE05FFD8327C101138507008320C102AD
:1017A0001301010367800000130101FD23261102CC
:1017B0002326A1002324B1008327C100232CF1009C
:1017C0008327810163960700737004306F00000067
:1017D00083278100639807008327810183A707047B
:1017E00063960700930710006F00800093070000C6
:1017F00063960700737004306F0000008327810137
:1018000083A7070463960700737004306F0000001D
:10181000EFE01FF793070500232AF10083278101DA
:1018200083A78703638A07028327810183A7C700F1
:101830002328F1008325810003258101EF00403337
:10184000832781010327010123A6E70093071000E6
:10185000232EF1006F008000232E01008327410119
:1018600013850700EFE01FF08327C10113850700F0
:101870008320C1021301010367800000130101FDF1
:10188000232611022326A1008327C10063960700A7
:10189000737004306F000000EF2090618327C10057
:1018A00083A78703232EF100EF2090648327C101D3
:1018B000138507008320C102130101036780000024
:1018C000130101FD232611022326A1008327C10055
:1018D000232EF1008327C101639607007370043043
:1018E0006F000000EF20D05C8327C10103A7C7036E
:1018F0008327C10183A78703B307F740232CF10097
:10190000EF20105F83278101138507008320C10228
:101910001301010367800000130101FE2326A100CB
:101920008327C10063960700737004306F000000C6
:101930008327C10083A78703232EF1008327C101DA
:10194000138507001301010267800000130101FDE8
:10195000232611022326A1008327C100232EF10094
:101960008327C10163960700737004306F00000085
:101970000325C101EF0040520325C101EF4050375C
:10198000130000008320C1021301010367800000DF
:10199000130101FF2326A1008327C10083A7C704E9
:1019A000138507001301010167800000130101FF87
:1019B0002326A1002324B1008327C100032781002F
:1019C00023A6E70413000000130101016780000053
:1019D000130101FF2326A1008327C10083C7070548
:1019E000138507001301010167800000130101FD49
:1019F000232611022326A1002324B1002322C100A3
:101A0000232E01008327C10083A7070463980702E0
:101A10008327C10083A70700639807128327C100AB
:101A200083A7470013850700EF20D034232EA100A1
:101A30008327C10023A207006F0000118327410004
:101A4000639407068327C10003A787008327C1008B
:101A500083A7070413860700832581001305070069
:101A6000EF40D03F8327C10003A787008327C10031
:101A700083A707043307F7008327C10023A4E700E7
:101A80008327C10003A787008327C10083A74700DE
:101A9000636CF70A8327C10003A707008327C100EF
:101AA00023A4E7006F00400A8327C10003A7C700F3
:101AB0008327C10083A707041386070083258100BD
:101AC00013050700EF4090398327C10003A7C70023
:101AD0008327C10083A70704B307F0403307F7004B
:101AE0008327C10023A6E7008327C10003A7C700FF
:101AF0008327C10083A707006372F7028327C10011
:101B000003A747008327C10083A70704B307F0405A
:101B10003307F7008327C10023A6E700032741000E
:101B2000930720006312F7028327C10083A787036E
:101B3000638C07008327C10083A787031387F7FF00
:101B40008327C10023ACE7028327C10083A7870353
:101B5000138717008327C10023ACE7028327C10145
:101B6000138507008320C102130101036780000071
:101B7000130101FE232E11002326A1002324B1000E
:101B80008327C10083A70704638207068327C10058
:101B900003A7C7008327C10083A707043307F70003
:101BA0008327C10023A6E7008327C10003A7C7003E
:101BB0008327C10083A74700636AF7008327C1001A
:101BC00003A707008327C10023A6E7008327C100DE
:101BD00003A7C7008327C10083A707041386070054
:101BE0009305070003258100EF40502713000000F4
:101BF0008320C1011301010267800000130101FE6F
:101C0000232E11002326A100EF20902A6F0000044C
:101C10008327C10083A74702638207048327C1008B
:101C20009387470213850700EF10D03F9307050005
:101C300063840700EF10D0788327C10083A787044F
:101C40001387F7FF8327C10023A4E7048327C1007C
:101C500083A78704E34EF0FA6F00800013000000B2
:101C60008327C1001307F0FF23A4E704EF205028C7
:101C7000EF2010246F0000048327C10083A7070111
:101C8000638207048327C100938707011385070038
:101C9000EF1050399307050063840700EF1050726E
:101CA0008327C10083A747041387F7FF8327C10059
:101CB00023A2E7048327C10083A74704E34EF0FA79
:101CC0006F008000130000008327C1001307F0FF9E
:101CD00023A2E704EF20D021130000008320C101DC
:101CE0001301010267800000130101FD2326110288
:101CF0002326A100EF20D01B8327C10083A78703E1
:101D00006398070093071000232EF1006F008000F6
:101D1000232E0100EF20D01D8327C101138507006A
:101D20008320C1021301010367800000130101FE3B
:101D30002326A1008327C100639607007370043037
:101D40006F0000008327C10083A787036398070003
:101D500093071000232EF1006F008000232E010056
:101D60008327C1011385070013010102678000006A
:101D7000130101FD232611022326A100EF20501399
:101D80008327C10003A787038327C10083A7C70355
:101D90006318F70093071000232EF1006F008000F6
:101DA000232E0100EF20D0148327C10113850700E3
:101DB0008320C1021301010367800000130101FEAB
:101DC0002326A1008327C1006396070073700430A7
:101DD0006F0000008327C10003A787038327C1008A
:101DE00083A7C7036318F70093071000232EF100A1
:101DF0006F008000232E01008327C1011385070097
:101E00001301010267800000130101FE2326A100D7
:101E10002324B100232E01006F00800617870300E2
:101E2000130787A98327C10193973700B307F700EA
:101E300083A7070063900704178703001307C7A74A
:101E40008327C10193973700B307F7000327810069
:101E500023A0E70017870300130707A68327C10104
:101E600093973700B307F7000327C10023A2E700C9
:101E70006F00C0018327C10193871700232EF10053
:101E80000327C10193077000E3FAE7F8130000008D
:101E90001301010267800000130101FE2326A10047
:101EA000232E01006F00C004178703001307C7A08B
:101EB0008327C10193973700B307F70083A7470033
:101EC0000327C1006310F702178703001307C79E9B
:101ED0008327C10193973700B307F70023A00700BA
:101EE0006F00C0018327C10193871700232EF100E3
:101EF0000327C10193077000E3F8E7FA130000001D
:101F00001301010267800000130101FD2326110265
:101F10002326A1002324B1002322C1008327C1006E
:101F2000232EF100EF20C0788327C10103A74704C7
:101F30009307F0FF6316F7008327C10123A207046C
:101F40008327C10103A787049307F0FF6316F700F7
:101F50008327C10123A40704EF2080798327C101CF
:101F600083A78703639E07008327C10193874702E6
:101F7000032641008325810013850700EF10007FB1
:101F80000325C101EFF09FC7130000008320C102A9
:101F90001301010367800000130101FC232E1102CD
:101FA000232EA100232CB1002328D1002326E100F9
:101FB0002324F100232201012320110193070600AD
:101FC000231BF1008327C10163960700737004305F
:101FD0006F0000000327C1009307400063F6E7008D
:101FE000737004306F000000835761018325410046
:101FF00013850700EF10D07E2324A10283278102DE
:102000006386071C8327810203A7070383566101A8
:10201000B70700409387F7FFB387F6009397270031
:10202000B307F7002322F1028327410293F7C7FF8A
:102030002322F1028327410293F7370063860700CA
:10204000737004306F00000083576101138707002D
:10205000832601000326C100832581010325810217
:10206000EF105041032601018325C10103254102E0
:10207000EFE00FF3130705008327810223A0E70099
:10208000832781006388070083278100032781025B
:1020900023A0E700EF20C06197E7010093878767DF
:1020A00083A707001387170097E7010093878766C8
:1020B00023A0E70097E701009387074D83A7070058
:1020C0006398070297E701009387074C0327810273
:1020D00023A0E70097E701009387C76303A70700E2
:1020E000930710006312F704EF10904B6F00C003CA
:1020F00097E701009387C76283A7070063960702EB
:1021000097E701009387474883A7070083A7C70283
:102110000327C100636AF70097E701009387C7466A
:102120000327810223A0E70097E701009387476018
:1021300083A707001387170097E701009387475F7E
:1021400023A0E70097E701009387875E03A70700B6
:102150008327810223A4E7048327810203A7C70200
:1021600097E701009387875B83A7070063FCE7007D
:102170008327810203A7C70297E701009387075AC5
:1021800023A0E7008327810203A7C7029307070064
:1021900093972700B387E7009397270017E701007D
:1021A0001307074A3387E700832781029387470095
:1021B0009385070013050700EFE00FF19307100068
:1021C0002326F102EF20C0526F00C0009307F0FFFA
:1021D0002326F1020327C102930710006318F702B8
:1021E00097E701009387C75383A70700638007021F
:1021F00097E701009387473983A7070083A7C702A2
:102200000327C10063F4E700EFE08FB88327C10222
:10221000138507008320C1031301010467800000B8
:10222000130101FD232611022326A100EF204048BF
:102230008327C100639A070097E701009387C7349B
:1022400083A707006F0080008327C100232EF100C1
:102250008327C1019387470013850700EFE00FFB39
:102260008327C10183A78702638A07008327C101EF
:102270009387870113850700EFE04FF98327C1019A
:10228000938747009385070017E501001305C545AF
:10229000EFE08FE397E701009387474683A70700A6
:1022A0001387170097E701009387474523A0E700AE
:1022B00097E701009387C74783A707001387170095
:1022C00097E701009387C74623A0E700EF2040422D
:1022D00097E701009387C74483A707006382070439
:1022E00097E701009387472A83A707000327C101C7
:1022F0006312F70297E701009387074483A707005B
:1023000063860700737004306F000000EFE04FA891
:102310006F000001EF20C039EF208001EF20403D29
:10232000130000008320C102130101036780000035
:10233000130101FD232611022326A1002324B1004D
:10234000232E01008327C1006396070073700430B9
:102350006F000000832781006396070073700430CC
:102360006F00000097E701009387073D83A70700F0
:1023700063860700737004306F000000EF00101DCB
:1023800097E701009387473983A70700232CF100C3
:102390008327C10083A7070003278100B307F70045
:1023A000232AF1008327C10083A7070003278101A7
:1023B0006376F7028327C10083A707000327410143
:1023C0006370F704032741018327810163FAE70261
:1023D00093071000232EF1006F0080028327C100B5
:1023E00083A70700032741016368F7000327410122
:1023F0008327810163F6E70093071000232EF10085
:102400008327C1000327410123A0E7008327C101DF
:102410006382070297E701009387071783A70700E6
:102420009387470013850700EFE04FDE0325410146
:10243000EF10502FEF00D0132328A10083270101B4
:1024400063940700EFE0CF94130000008320C102E3
:102450001301010367800000130101FD232611020F
:102460002326A100232E01008327C10063800706D5
:1024700097E701009387472C83A70700638607002F
:10248000737004306F000000EF00500C97E70100FC
:102490009387872883A707000327C100B307F700A6
:1024A000232CF10097E701009387070E83A707000D
:1024B0009387470013850700EFE04FD5032581017F
:1024C000EF105026EF00D00A232EA1008327C10170
:1024D00063940700EFE0CF8B130000008320C1025C
:1024E0001301010367800000130101FD232611027F
:1024F0002326A1008327C100232CF100832781011B
:1025000063960700737004306F00000097E70100C6
:102510009387870783A70700032781016316F700C6
:10252000232E01006F00400AEF20801883278101CD
:1025300083A74701232AF100EF20801B97E70100C2
:102540009387C71883A7070003274101630CF7008F
:1025500097E701009387C71783A707000327410167
:102560006318F70093072000232EF1006F00C005C9
:102570000327410197E70100938787186314F70247
:102580008327810183A787026398070093073000A0
:10259000232EF1006F00400393072000232EF1004B
:1025A0006F0080020327410197E701009387C7135B
:1025B0006318F70093074000232EF1006F00C0005E
:1025C00093071000232EF1008327C1011385070014
:1025D0008320C1021301010367800000130101FD84
:1025E000232611022326A100EF20800C8327C1009F
:1025F000639A070097E70100938707F983A707000D
:102600006F0080008327C100232EF1008327C101C2
:1026100083A7C702232CF100EF20800D83278101BF
:10262000138507008320C1021301010367800000A6
:10263000130101FD232611022326A100EFE04F9490
:1026400093070500232EF1008327C100639A07003A
:1026500097E70100938747F383A707006F00800087
:102660008327C100232CF1008327810183A7C702A0
:10267000232AF1008327C10113850700EFE08F8E25
:1026800083274101138507008320C1021301010341
:1026900067800000130101FD232611022326A100FB
:1026A0002324B100232E010003278100930740005B
:1026B00063F6E700737004306F00000003278100A9
:1026C0009307400063F6E700930740002324F100DE
:1026D000EF10107E8327C100639A070097E701007F
:1026E000938787EA83A707006F0080008327C100D4
:1026F000232CF1008327810183A70705232AF100FA
:102700000327410183278100630EF7160327810009
:102710008327410163FEE70297E701009387C7E63D
:1027200083A70700032781016302F70497E70100ED
:10273000938787E583A7070083A7C7020327810044
:102740006366F70293071000232EF1006F0000026A
:1027500097E70100938747E383A7070003278101D9
:102760006316F70093071000232EF10083278101E1
:1027700083A7C7022328F1008327810103A7070548
:102780008327810183A7C7026318F700832781018C
:102790000327810023A6E702832781010327810005
:1027A00023A8E7048327810183A7870163CC07005F
:1027B00013075000832781003307F74083278101E7
:1027C00023ACE7008327810183A64701032701018A
:1027D0009307070093972700B387E7009397270095
:1027E00017E701001307C7E5B387E7006396F60014
:1027F000930710006F00800093070000638C0706AA
:10280000832781019387470013850700EFE00FA01E
:102810008327810103A7C70297E70100938707F089
:1028200083A7070063FCE7008327810103A7C70292
:1028300097E70100938787EE23A0E70083278101B4
:1028400003A7C7029307070093972700B387E70002
:102850009397270017E70100130787DE3387E70008
:10286000832781019387470093850700130507009D
:10287000EFE08F850327C101930710006314F70071
:10288000EFD01FD1EF10D066130000008320C102EB
:102890001301010367800000130101FD23261102CB
:1028A0002326A100EF10D0608327C100639A0700A0
:1028B00097E70100938747CD83A707006F0080004B
:1028C0008327C100232EF1008327C101938747008E
:1028D00013850700EFE08F938327C10183A7870249
:1028E000638A07008327C101938787011385070047
:1028F000EFE0CF918327C1019387470093850700BD
:1029000017E501001305C5DFEFD01FFCEF10505E87
:1029100097E70100938747C783A707000327C101F3
:102920006314F70697E70100938787DF83A7070003
:102930006382070297E70100938707E083A70700F8
:1029400063860700737004306F000000EFD05FC42F
:102950006F00400597E70100938787DA03A7070018
:1029600097E70100938707DB83A70700631AF70047
:1029700097E70100938747C123A007006F008002FB
:10298000EF0090286F00000297E70100938747D976
:1029900083A7070063880700EF109051EF105019CC
:1029A000EF101055130000008320C1021301010332
:1029B00067800000130101FE2326A100232E0100E1
:1029C0008327C100232CF1008327C10063960700F1
:1029D000737004306F0000008327810103A7470153
:1029E00097E701009387C7D16316F700930710009C
:1029F0006F00800093070000638E07028327810128
:102A000003A7870297E701009387C7CC6304F70207
:102A10008327810183A7870263960700930710002D
:102A20006F00800093070000638607009307100083
:102A3000232EF1008327C101138507001301010232
:102A400067800000130101FD232611022326A10047
:102A50008327C100232EF1008327C100639607005E
:102A6000737004306F0000008327C1016384070C7A
:102A700097E70100938747B183A707000327C101A8
:102A8000630AF70AEF10D0420325C101EFF09FF26D
:102A90001307050093071000631CF7088327C10183
:102AA0009387470013850700EFD05FF68327C101A6
:102AB00003A7C70297E70100938747C683A70700CC
:102AC00063FCE7008327C10103A7C70297E7010062
:102AD0009387C7C423A0E7008327C10103A7C702C8
:102AE0009307070093972700B387E7009397270082
:102AF00017E701001307C7B43387E7008327C10135
:102B0000938747009385070013050700EFD0DFDBAD
:102B10008327C10103A7C70297E701009387C7A6D0
:102B200083A7070083A7C7026364F700EFD05FA6FF
:102B3000EF10103C130000008320C10213010103B9
:102B400067800000130101FD232611022326A10046
:102B5000232E01008327C100232CF1008327C1000D
:102B600063960700737004306F000000EFD05FC100
:102B700093070500232AF10003258101EFF09FE36D
:102B800013070500930710006314F70C97E7010083
:102B9000938787BA83A707006390070A8327810179
:102BA00003A7C70297E701009387079E83A7070043
:102BB00083A7C7026366F70093071000232EF10076
:102BC000832781019387470013850700EFD01FE417
:102BD0008327810103A7C70297E70100938707B402
:102BE00083A7070063FCE7008327810103A7C702CF
:102BF00097E70100938787B223A0E700832781012D
:102C000003A7C7029307070093972700B387E7003E
:102C10009397270017E70100130787A23387E70080
:102C200083278101938747009385070013050700D9
:102C3000EFD09FC96F00C00183278101938787016F
:102C40009385070017E501001305C5A8EFD0DFC77E
:102C50008327410113850700EFD0DFB08327C1012F
:102C6000138507008320C102130101036780000060
:102C7000130101FE232E1100930800001308000029
:102C8000930700001307000093060000130600409E
:102C900097D501009385053717150000130505FB2F
:102CA000EFF08FAF2326A1000327C1009307100088
:102CB0006316F700EF20C03A2326A1000327C100C6
:102CC00093071000631EF7027370043097E701004A
:102CD000938747A61307F0FF23A0E70097E70100BB
:102CE000938707A41307100023A0E70097E70100CC
:102CF000938787A223A00700EFD0CFEE6F0040019B
:102D00008327C10063960700737004306F000000D2
:102D1000130000008320C10113010102678000003D
:102D2000130101FF232611007370043097E701009F
:102D30009387079F23A00700EFD00FFD130000002B
:102D40008320C100130101016780000097E70100A3
:102D50009387879E83A707001387170097E70100D3
:102D60009387879D23A0E700130000006780000081
:102D7000130101FE232E11002326010097E7010015
:102D80009387879B83A707006396070073700430BF
:102D90006F000000EF10D01197E701009387C799EB
:102DA00083A707001387F7FF97E701009387C7986A
:102DB00023A0E70097E701009387079883A7070000
:102DC0006394071697E701009387C79483A70700CA
:102DD000638C07146F00800C97E701009387878F3F
:102DE00083A7C70083A7C7002324F100832781009E
:102DF0009387870113850700EFD05FC18327810088
:102E00009387470013850700EFD05FC083278100B9
:102E100003A7C70297E701009387479083A707009E
:102E200063FCE7008327810003A7C70297E701003F
:102E30009387C78E23A0E7008327810003A7C702DB
:102E40009307070093972700B387E700939727001E
:102E500017D701001307C77E3387E7008327810058
:102E6000938747009385070013050700EFD0DFA580
:102E70008327810003A7C70297D701009387C770F4
:102E800083A7070083A7C702636AF70097E70100DB
:102E9000938787891307100023A0E70097E70100B5
:102EA0009387478383A70700E39807F297E701001A
:102EB0009387478783A70700638807046F00C003D1
:102EC000EF00002B93070500638A070097E70100D6
:102ED000938787851307100023A0E70097E7010079
:102EE0009387478483A707001387F7FF97E70100BD
:102EF0009387478323A0E70097E7010093878782A2
:102F000083A70700E39E07FA97E701009387C7812D
:102F100003A70700930710006318F700930710003A
:102F20002326F100EFD0CFE6EF10807C8327C1008D
:102F3000138507008320C10113010102678000008F
:102F4000130101FE232E1100EF10807697D70100A8
:102F50009387877C83A707002326F100EF10407931
:102F60008327C100138507008320C10113010102DB
:102F700067800000130101FE232E1100EFD05F8057
:102F8000930705002326F10097D701009387C778A0
:102F900083A707002324F1008327C10013850700BE
:102FA000EFD04FFC83278100138507008320C101E8
:102FB000130101026780000097D70100938787758E
:102FC00083A707001385070067800000130101FD38
:102FD000232611022326A1002324B1002322C100AD
:102FE000232E010093075000232CF100EFF01FD691
:102FF00097D701009387077283A7070003278100F3
:10300000636CF714832781019387F7FF232CF1006A
:103010008327C101939757000327C100B306F70028
:10302000032781019307070093972700B387E700E1
:103030009397270017D7010013078760B387E7002E
:10304000130610009385070013850600EF10800417
:10305000130705008327C101B387E700232EF10082
:1030600083278101E39007FA8327C10193975700D3
:103070000327C1003307F70097D70100938707653F
:1030800083A7070013062000938507001305070098
:10309000EF104000130705008327C101B387E70045
:1030A000232EF1008327C101939757000327C10006
:1030B0003307F70097D701009387876183A707003D
:1030C000130620009385070013050700EF00907C8E
:1030D000130705008327C101B387E700232EF10002
:1030E0008327C101939757000327C100B307F70057
:1030F0001306400097D501009385055F13850700EF
:10310000EF005079130705008327C101B387E7005B
:10311000232EF1008327C101939757000327C10095
:10312000B307F7001306300097D501009385455D7E
:1031300013850700EF001076130705008327C101F0
:10314000B387E700232EF100832741006386070041
:103150008327410023A00700EFF09FC18327C1010F
:10316000138507008320C10213010103678000005B
:10317000130101FD23261102232E010097D7010020
:103180009387875B83A70700639C072297D701007B
:103190009387875883A707001387170097D70100E5
:1031A0009387875723A0E70097D701009387C756D7
:1031B00083A70700232CF10083278101639C070666
:1031C00097D701009387875083A7070083A707003D
:1031D00063860700737004306F00000097D701000A
:1031E0009387C74E83A70700232AF10097D70100D2
:1031F0009387074E03A7070097D701009387074DD2
:1032000023A0E70097D701009387874C032741014C
:1032100023A0E70097D701009387475183A70700B2
:103220001387170097D701009387475023A0E70023
:10323000EF10001097D701009387C74F83A70700AF
:1032400003278101636CF71297D701009387074822
:1032500083A7070083A70700639607009307100062
:103260006F00800093070000638C070097D7010070
:103270009387474C1307F0FF23A0E7006F0000106F
:1032800097D701009387874483A7070083A7C700C8
:1032900083A7C7002328F1008327010183A74700E4
:1032A0002326F100032781018327C100637CF700F7
:1032B00097D70100938707480327C10023A0E700A1
:1032C0006F00C00B83270101938747001385070018
:1032D000EFD0CFF38327010183A78702638A07001A
:1032E000832701019387870113850700EFD00FF231
:1032F0008327010103A7C70297D7010093870742DD
:1033000083A7070063FCE7008327010103A7C70227
:1033100097D701009387874023A0E7008327010107
:1033200003A7C7029307070093972700B387E70017
:103330009397270017D70100130787303387E700DB
:103340008327010193874700938507001305070032
:10335000EFD08FD78327010103A7C70297D70100BA
:103360009387872283A7070083A7C702E36EF7EC42
:1033700093071000232EF1006FF01FED97D7010087
:103380009387872083A7070003A7C70297D601006A
:103390009386062B9307070093972700B387E700D0
:1033A00093972700B387F60003A707009307100041
:1033B00063F6E70293071000232EF1006F0000026E
:1033C00097D701009387073683A707001387170055
:1033D00097D701009387073523A0E70097D701000F
:1033E0009387873483A7070063860700930710003D
:1033F000232EF1008327C101138507008320C1021A
:103400001301010367800000130101FE232E110048
:1034100097D701009387473283A70700638C070083
:1034200097D70100938747301307100023A0E700C8
:103430006F00C01897D701009387072F23A00700BC
:1034400097D701009387471483A7070083A7070333
:103450002326F100B7A7A5A59387575A2324F10087
:103460008327C10083A70700032781006310F704A7
:103470008327C1009387470083A7070003278100A4
:103480006316F7028327C1009387870083A707008D
:1034900003278100631CF7008327C1009387C700BF
:1034A00083A70700032781006302F70697D701006F
:1034B0009387870D03A7070097D701009387C70C51
:1034C00083A7070093874703938507001305070029
:1034D000EF40C00E6F00800397D701009387072449
:1034E00083A7070063960700737004306F00000025
:1034F00097D701009387872283A707001387F7FFD9
:1035000097D701009387872123A0E70097D7010071
:103510009387C72003A7070097D60100938646121A
:103520009307070093972700B387E7009397270037
:10353000B387F60083A70700E38007FA97D7010057
:103540009387C71D03A707009307070093972700DA
:10355000B387E7009397270017D701001307470E9B
:10356000B387E7002322F1008327410083A74700A8
:1035700003A747008327410023A2E70083274100D8
:1035800003A747008327410093878700631CF70048
:103590008327410083A7470003A7470083274100F3
:1035A00023A2E7008327410083A7470003A7C700A2
:1035B00097D70100938747FD23A0E7001300000081
:1035C0008320C1011301010267800000130101FD86
:1035D000232611022326A1002324B1008327C10042
:1035E00063960700737004306F00000097D70100E6
:1035F000938787F983A7070093878701938507003F
:103600000325C100EFD00FB497D701009387C7F708
:1036100083A707009387470013850700EFD00FBFEC
:10362000032781009307F0FF6314F70297D7010087
:10363000938787F583A70700938747009385070043
:1036400017D501001305C50BEFD00FA86F0040027E
:1036500097D701009387470C83A7070003278100B2
:10366000B307F700232EF1000325C101EF00900BF3
:10367000130000008320C1021301010367800000D2
:10368000130101FD232611022326A1002324B100EA
:103690002322C1008327C1006396070073700430A2
:1036A0006F00000097D701009387070983A70700E1
:1036B00063960700737004306F00000097D7010015
:1036C000938787EC83A70700832681003707008054
:1036D00033E7E60023ACE70097D701009387C7EAFA
:1036E00083A7070093878701938507000325C100FF
:1036F000EFD08F9D97D70100938707E983A7070035
:103700009387470013850700EFD04FB00327410090
:103710009307F0FF6314F70297D701009387C7E67A
:1037200083A70700938747009385070017D50100FB
:10373000130505FDEFD04F996F00400297D70100A8
:10374000938787FD83A7070003274100B307F7008E
:10375000232EF1000325C101EF00C07C13000000FF
:103760008320C1021301010367800000130101FDE2
:10377000232611022326A1002324B1002322C10005
:103780008327C10063960700737004306F00000048
:1037900097D70100938747DF83A7070093878701A7
:1037A000938507000325C100EFD00F9297D7010042
:1037B000938787DD83A7070093874700138507005A
:1037C000EFD0CFA403274100930710006314F70242
:1037D00097D70100938747DB83A7070093874700AC
:1037E0009385070017D50100130585F1EFD0CF8D24
:1037F0006F00400297D70100938707F283A7070065
:1038000003278100B307F700232EF1000325C10130
:10381000EF004071130000008320C1021301010377
:1038200067800000130101FD232611022326A10059
:103830008327C10083A7C70083A7C700232CF100FB
:103840008327810163960700737004306F000000C6
:10385000832781019387870113850700EFD00F9B92
:1038600097D70100938747ED83A70700639E07065C
:10387000832781019387470013850700EFD00F99B5
:103880008327810103A7C70297D70100938707E920
:1038900083A7070063FCE7008327810103A7C70212
:1038A00097D70100938787E723A0E700832781014B
:1038B00003A7C7029307070093972700B387E70082
:1038C0009397270017D70100130787D73387E7009F
:1038D000832781019387470093850700130507001D
:1038E000EFC09FFE6F00C00183278101938787018E
:1038F0009385070017D501001305C5DDEFC0DFFC78
:103900008327810103A7C70297D701009387C7C701
:1039100083A7070083A7C70263F0E702930710009D
:10392000232EF10097D70100938707E013071000BB
:1039300023A0E7006F008000232E01008327C10130
:10394000138507008320C102130101036780000073
:10395000130101FD232611022326A1002324B10017
:1039600097D70100938747DD83A707006396070079
:10397000737004306F00000003278100B7070080D8
:103980003367F7008327C10023A0E7008327C10026
:1039900083A7C700232CF1008327810163960700CA
:1039A000737004306F0000000325C100EFD00F8654
:1039B000832781019387470013850700EFD00F8588
:1039C0008327810103A7C70297D70100938707D5F3
:1039D00083A7070063FCE7008327810103A7C702D1
:1039E00097D70100938787D323A0E700832781011E
:1039F00003A7C7029307070093972700B387E70041
:103A00009397270017D70100130787C33387E70071
:103A100083278101938747009385070013050700DB
:103A2000EFC09FEA8327810103A7C70297D7010050
:103A3000938787B583A7070083A7C70263F0E702D0
:103A400093071000232EF10097D701009387C7CD6D
:103A50001307100023A0E7006F008000232E010051
:103A60008327C101138507008320C10213010103CD
:103A700067800000130101FF2326A1008327C100F6
:103A800063960700737004306F00000097D7010041
:103A90009387C7C903A707008327C10023A0E700B6
:103AA00097D70100938747C703A707008327C10063
:103AB00023A2E7001300000013010101678000004A
:103AC000130101FD232611022326A1002324B100A6
:103AD0008327C10063960700737004306F000000F5
:103AE0008327810063960700737004306F00000025
:103AF000EF00103C97D70100938707C283A7070008
:103B0000232CF1008327810003A707009307F0FF10
:103B10006316F700232E01006F0000098327C10000
:103B200003A7070097D70100938747C083A7070023
:103B30006300F7028327C10083A7470003278101A1
:103B40006368F70093071000232EF1006F00C00593
:103B50008327C10083A74700032781013307F7406C
:103B60008327810083A70700637CF70283278100F6
:103B700003A707008327C10083A64700832781018D
:103B8000B387F6403307F7008327810023A0E700BF
:103B90000325C100EFF01FEE232E01006F00C000CF
:103BA00093071000232EF100EF0090348327C1010A
:103BB000138507008320C102130101036780000001
:103BC00097D70100938747B61307100023A0E7009B
:103BD0001300000067800000130101FE2326A100EE
:103BE0008327C100638E07008327C100232CF100C7
:103BF0008327810183A7C704232EF1006F00800073
:103C0000232E01008327C101138507001301010240
:103C100067800000130101FE2326A1002324B100C8
:103C20008327C100638C07008327C100232EF10086
:103C30008327C1010327810023A6E70413000000A6
:103C40001301010267800000130101FE232E110001
:103C50002326A100EF00002197D701009387479EFC
:103C600003A7070093071000E3F6E7FEEFC05F929B
:103C70006FF05FFE130101FC232E1102232EA10021
:103C8000232CB100232AC1002328D1009307070069
:103C90002317F100232601026F004004032781014E
:103CA0008327C102B307F70003C707008326C101BA
:103CB0008327C102B387F600238AE7020327810125
:103CC0008327C102B307F70083C707006380070299
:103CD0008327C102938717002326F1020327C1021D
:103CE0009307F000E3FCE7FA6F0080001300000088
:103CF0008327C101A38107040327410193074000E3
:103D000063F6E70093074000232AF1008327C101EF
:103D10000327410123A6E7028327C10103274101AD
:103D200023A8E7048327C10123AA07048327C1012D
:103D30009387470013850700EFC05FB78327C10152
:103D40009387870113850700EFC05FB68327C10102
:103D50000327C10123A8E70013075000832741016F
:103D60003307F7408327C10123ACE7008327C10154
:103D70000327C10123A2E7028327C10123A207046D
:103D80008327C10123AC07048327C10123AE0704A5
:103D9000130000008320C1031301010467800000A9
:103DA000130101FE232E1100232601006F00800362
:103DB0000327C1009307070093972700B387E70005
:103DC0009397270017D7010013078787B387E7006A
:103DD00013850700EFC01FA88327C1009387170032
:103DE0002326F1000327C10093074000E3F2E7FC1C
:103DF00017D501001305058BEFC0DFA517D501000E
:103E00001305858BEFC01FA517D501001305858C01
:103E1000EFC05FA417D501001305058DEFC09FA368
:103E200017D501001305C58DEFC0DFA297D701009C
:103E30009387C78917D701001307C78623A0E70018
:103E400097D701009387C78817D701001307C78644
:103E500023A0E700130000008320C1011301010229
:103E600067800000130101FE232E11006F008009FE
:103E7000EFE0DFED97D701009387078783A707005F
:103E800093B7170093F7F70F2326F100EFE05FEEEB
:103E90008327C10063980706EF00900197D70100C0
:103EA0009387878483A7C70083A7C7002324F100D3
:103EB000832781009387470013850700EFC01FB554
:103EC00097D701009387078583A707001387F7FF1C
:103ED00097D701009387078423A0E70097D70100B5
:103EE0009387C78183A707001387F7FF97D7010040
:103EF0009387C78023A0E700EF00807F0325810020
:103F0000EF00C03F97C701009387477F83A7070053
:103F1000E39007F6130000008320C10113010102A2
:103F200067800000130101FE232E11002326A1004B
:103F300097C701009387476583A707000327C10040
:103F400023A2E70097C701009387077D83A7070097
:103F50000327C1006378F70297C70100938747776B
:103F600003A7070097C701009387076283A707008D
:103F7000938747009385070013050700EFC09F9CB8
:103F80006F00000597C701009387477403A70700D8
:103F900097C701009387475F83A707009387470070
:103FA0009385070013050700EFC0DF9997C701004D
:103FB0009387477883A707000327C100637AF70038
:103FC00097C70100938707770327C10023A0E70065
:103FD000130000008320C10113010102678000006B
:103FE000130101FD23261102930705002324B100CC
:103FF0002317F10083278100639E07008357E100A8
:104000009397270013850700EF20C02E9307050024
:104010006F00800083278100232CF100832781011A
:10402000638A070213050006EF20C02C232EA1008F
:104030008327C101638A07008327C1010327810108
:1040400023A8E7026F00400103258101EF20404AC9
:104050006F008000232E01008327C10163820702C5
:104060008327C10103A707038357E1009397270024
:10407000138607009305500A13050700EF20006A16
:104080008327C101138507008320C10213010103A7
:1040900067800000130101FC232E1102232C8102F2
:1040A0002326A1002324B1002322C10023260102DC
:1040B0008327810083A707006388071C832781006B
:1040C0002324F1028327810283A7470003A7470027
:1040D0008327810223A2E7008327810203A74700E9
:1040E0008327810293878700631CF700832781025F
:1040F00083A7470003A747008327810223A2E70085
:104100008327810283A7470083A7C7002322F102E8
:10411000832781002320F1028327010283A7470020
:1041200003A747008327010223A2E7008327010298
:1041300003A747008327010293878700631CF700CA
:104140008327010283A7470003A7470083270102B3
:1041500023A2E7008327010283A7470083A7C700A4
:10416000232EF1008327C102939757000327C10034
:10417000B307F7000327C10123A0E7008327C1028B
:10418000939757000327C100B307F7000327C10126
:104190001307470323A2E7008327C1029397570021
:1041A0000327C100B307F7000327C10103278704D2
:1041B00023A4E7008327C102939757000327C10078
:1041C000B307F7000327410023A6E7008327C102B6
:1041D000939757000327C100B307F7000327C101D6
:1041E0000327C70223A8E7000327410093073000F5
:1041F0006314F7028327C10183A78702638E070038
:104200008327C102939757000327C100B307F70024
:104210001307200023A6E7008327C10293975700C6
:104220000327C100B307F7000327C10103270705D0
:1042300023AAE7008327C102939757000327C100F1
:10424000B307F70023AC07008327C10183A6070348
:104250008327C102939757000327C1003304F70057
:1042600013850600EF00C00393070500231EF4002A
:104270008327C102938717002326F1020327C10178
:1042800083274102E316F7E88327C102138507005D
:104290008320C1030324810313010104678000000C
:1042A000130101FE2326A100232E01006F00C0018F
:1042B0008327C100938717002326F1008327C101BC
:1042C00093871700232EF1008327C10003C707003F
:1042D0009307500AE30EF7FC8327C10193D7270009
:1042E000232EF1008327C1019397070193D707017C
:1042F000138507001301010267800000130101FE0E
:10430000232E11002326A1008327C10083A70703C2
:1043100013850700EF20C01D0325C100EF20401DBD
:10432000130000008320C101130101026780000017
:10433000130101FF97C701009387473983A707003F
:1043400083A7070063960700930710006F008000A3
:1043500093070000638C070097C701009387873D90
:104360001307F0FF23A0E7006F00000397C70100C9
:104370009387C73583A7070083A7C70083A7C70014
:104380002326F1008327C10003A7470097C7010038
:104390009387473A23A0E7001300000013010101AF
:1043A00067800000130101FF97C701009387C71DB5
:1043B00083A707002326F1008327C1001385070088
:1043C0001301010167800000130101FF97C701007D
:1043D0009387073583A707006398070093071000AA
:1043E0002326F1006F00400297C701009387C7346E
:1043F00083A7070063980700930720002326F10096
:104400006F008000232601008327C1001385070069
:104410001301010167800000130101FD2326110231
:104420002326A1008327C100232EF1008327C1008A
:10443000638A07128327C10103A7C70297C7010038
:104440009387871483A7070083A7C702637CF710AD
:104450008327C10183A7870163C2070297C70100B1
:104460009387871283A7070083A7C702130750000B
:104470003307F7408327C10123ACE7008327C1013D
:1044800083A647018327C10103A7C702930707003B
:1044900093972700B387E7009397270017C701007A
:1044A0001307071AB387E7006396F6009307100017
:1044B0006F00800093070000638A07088327C1010B
:1044C0009387470013850700EFC04FD497C70100BB
:1044D0009387870B83A7070003A7C7028327C10120
:1044E00023A6E7028327C10103A7C70297C70100DC
:1044F0009387C72283A7070063FCE7008327C101D6
:1045000003A7C70297C701009387472123A0E700AD
:104510008327C10103A7C7029307070093972700CA
:10452000B387E7009397270017C7010013074711C8
:104530003387E7008327C1019387470093850700EE
:1045400013050700EFC04FB86F00C00197C7010007
:104550009387870383A7070003A7C7028327C101A7
:1045600023A6E702130000008320C1021301010308
:1045700067800000130101FD232611022326A100FC
:104580008327C100232CF100232E01008327C100C3
:104590006386071097C70100938707FF83A707006B
:1045A000032781016306F700737004306F00000079
:1045B0008327810183A74705639607007370043042
:1045C0006F0000008327810183A747051387F7FF4A
:1045D0008327810123AAE7048327810103A7C70258
:1045E0008327810183A70705630AF70A83278101CF
:1045F00083A747056394070A8327810193874700B0
:1046000013850700EFC08FC08327810103A707052B
:104610008327810123A6E7028327810183A7C7029D
:10462000130750003307F7408327810123ACE700CD
:104630008327810103A7C70297C701009387070E4D
:1046400083A7070063FCE7008327810103A7C70254
:1046500097C701009387870C23A0E7008327810178
:1046600003A7C7029307070093972700B387E700C4
:104670009397270017C70100130787FC3387E700CC
:10468000832781019387470093850700130507005F
:10469000EFC08FA393071000232EF1008327C101E1
:1046A000138507008320C102130101036780000006
:1046B0007370043097C701009387870683A70700AC
:1046C0006384070297C70100938707EC83A707005D
:1046D00003A747041307170023A2E70497C70100A5
:1046E000938787EA83A70700130000006780000014
:1046F00097C701009387C70283A707006384070455
:1047000097C70100938747E883A7070083A747045B
:10471000638A070297C70100938707E783A707000B
:1047200003A747041307F7FF23A2E70497C7010075
:10473000938787E583A7070083A74704639407004F
:10474000736004301300000067800000130101FF54
:1047500097C70100938747E383A7070083A78701D3
:104760002326F10097C70100938707E283A707007C
:1047700003A7C70297C70100938707E183A7070034
:10478000930650003387E64023ACE7008327C1003F
:1047900013850700130101016780000097C701001E
:1047A000938787DE83A70700638E070097C7010002
:1047B000938787DD83A7070003A747051307170023
:1047C00023AAE70497C70100938707DC83A70700A4
:1047D0001385070067800000130101FD23261102E5
:1047E0002326A1002324B100EFF09FEC97C701001E
:1047F000938787D983A7070083A787056396070850
:1048000097C70100938747D883A7070013071000B5
:1048100023AEE704832781006388070697C701005A
:10482000938787D683A707009387470013850700E0
:10483000EFC0CF9D032781009307F0FF6314F702B9
:1048400097C70100938747D483A707009387470042
:104850009385070017C50100130585EAEFC0CF86D1
:104860006F00400297C70100938707EB83A70700FB
:1048700003278100B307F700232EF1000325C101B0
:10488000EFF04FEAEFB0DFD0EFF09FE6EFF05FE23E
:1048900097C70100938747CF83A7070083A78705A2
:1048A000232CF10083278101638C07028327C10039
:1048B000638C070097C70100938707CD83A7070084
:1048C00023AC07046F00C00197C701009387C7CBD3
:1048D00083A7070003A787051307F7FF23ACE704A7
:1048E00097C70100938747CA83A7070023AE070431
:1048F000EFF01FE083278101138507008320C102A9
:104900001301010367800000130101FD232611023A
:104910002326A1002324B1002322C1002320D1009B
:10492000EFF01FD997C70100938707C683A7070039
:1049300003A7C705930720006306F70A97C701007E
:10494000938787C483A7070083A687050327C10031
:104950001347F7FF33F7E60023ACE70497C70100DE
:10496000938787C283A707001307100023AEE704CD
:10497000832701006388070697C701009387C7C094
:1049800083A707009387470013850700EFC00F88B0
:10499000032701009307F0FF6314F70297C7010094
:1049A000938787BE83A707009387470093850700F7
:1049B00017C501001305C5D4EFB01FF16F00400209
:1049C00097C70100938747D583A7070003270100F6
:1049D000B307F700232CF10003258101EFF08FD4FA
:1049E000EFB01FBBEFF0DFD0EFF09FCC832741008B
:1049F000638E070097C70100938707B983A7070055
:104A000003A787058327410023A0E70097C701007C
:104A1000938787B783A7070003A7C70593071000ED
:104A20006316F700232E01006F00C00297C7010034
:104A3000938787B583A7070083A68705032781008F
:104A40001347F7FF33F7E60023ACE70493071000A2
:104A5000232EF10097C70100938707B383A70700B0
:104A600023AE0704EFF0DFC88327C10113850700D9
:104A70008320C1021301010367800000130101FDBF
:104A8000232611022326A1002324B1002322C100E2
:104A90002320D10093071000232EF1008327C100AB
:104AA00063960700737004306F0000008327C10015
:104AB000232CF100EFF0DFBF83270100638A07009A
:104AC0008327810103A787058327010023A0E7002F
:104AD0008327810183A7C705232AF100832781014A
:104AE0001307200023AEE70403274100930740008B
:104AF00063ECE708832741001397270097B701006D
:104B00009387C750B307F70003A7070097B70100C3
:104B10009387C74FB307F70067800700832781019A
:104B200003A78705832781003367F7008327810167
:104B300023ACE7046F0040058327810183A7870525
:104B4000138717008327810123ACE7046F00C0039C
:104B5000832781010327810023ACE7046F00C00293
:104B60000327410193072000630AF700832781018F
:104B70000327810023ACE7046F000001232E01000E
:104B80006F0080001300000003274101930710000D
:104B90006316F70A8327810193874700138507006F
:104BA000EFB0DFE68327810103A7C70297C70100A3
:104BB0009387C7B683A7070063FCE70083278101BB
:104BC00003A7C70297C70100938747B523A0E70053
:104BD0008327810103A7C702930707009397270044
:104BE000B387E7009397270017C70100130747A56E
:104BF0003387E70083278101938747009385070068
:104C000013050700EFB05FCC8327810183A78702DC
:104C100063860700737004306F00000083278101F2
:104C200003A7C70297C701009387079683A70700CA
:104C300083A7C70263F4E700EFB09F95EFF05FAB87
:104C40008327C101138507008320C10213010103DB
:104C500067800000130101FC232E1102232EA10006
:104C6000232CB100232AC1002328D1002326E100F0
:104C7000930710002326F1028327C10163960700E2
:104C8000737004306F0000008327C1012324F102F8
:104C9000EFB01FAF930705002322F1028327010124
:104CA000638A07008327810203A787058327010101
:104CB00023A0E7008327810283A7C7052320F102F1
:104CC000832781021307200023AEE7040327410155
:104CD0009307400063ECE7088327410113972700FF
:104CE00097B701009387C733B307F70003A70700FF
:104CF00097B701009387C732B307F70067800700B3
:104D00008327810203A78705832781013367F70083
:104D10008327810223ACE7046F00400583278102CB
:104D200083A78705138717008327810223ACE70435
:104D30006F00C003832781020327810123ACE704AE
:104D40006F00C0020327010293072000630AF700E7
:104D5000832781020327810123ACE7046F00000150
:104D6000232601026F0080001300000003270102C8
:104D7000930710006314F70E8327810283A787022D
:104D800063860700737004306F00000097C701004E
:104D90009387879A83A70700639E0706832781026C
:104DA0009387470013850700EFB05FC68327810212
:104DB00003A7C70297C701009387479683A70700F9
:104DC00063FCE7008327810203A7C70297C701009E
:104DD0009387C79423A0E7008327810203A7C70214
:104DE0009307070093972700B387E700939727005F
:104DF00017C701001307C7843387E70083278102A1
:104E0000938747009385070013050700EFB0DFABDA
:104E10006F00C00183278102938787019385070074
:104E200017C501001305058BEFB01FAA8327810268
:104E300003A7C70297B701009387077583A70700E9
:104E400083A7C70263FCE7008327C10063880700CC
:104E50008327C1001307100023A0E7008327410226
:104E600013850700EFB01F908327C1021385070049
:104E70008320C1031301010467800000130101FDB9
:104E8000232611022326A1002324B1008327C10079
:104E900063960700737004306F0000008327C10021
:104EA000232EF100EFB0DF8D93070500232CF100D6
:104EB0008327C10183A7C705232AF1008327C101E6
:104EC0001307200023AEE7048327C10183A78705CA
:104ED000138717008327C10123ACE704032741018F
:104EE000930710006314F70E8327C10183A787027D
:104EF00063860700737004306F00000097C70100DD
:104F00009387878383A70700639E07068327C101D2
:104F10009387470013850700EFB05FAF8327C10178
:104F200003A7C70297B701009387477F83A70700AE
:104F300063FCE7008327C10103A7C70297B70100FD
:104F40009387C77D23A0E7008327C10103A7C7027A
:104F50009307070093972700B387E70093972700ED
:104F600017B701001307C76D3387E7008327C10117
:104F7000938747009385070013050700EFB0DF9480
:104F80006F00C0018327C1019387870193850700C4
:104F900017B5010013050574EFB01F938327C101F6
:104FA00003A7C70297B701009387075E83A707008F
:104FB00083A7C70263FCE70083278100638807009B
:104FC000832781001307100023A0E70083278101B6
:104FD00013850700EFB00FF9130000008320C10212
:104FE0001301010367800000130101FD2326110254
:104FF0002326A1008327C100232CF10083278101F0
:10500000639A070097B701009387075883A70700A3
:105010006F00800083278101232CF100EFF04FE91E
:105020008327810103A7C70593072000631CF700AE
:105030008327810123AE070493071000232EF1007C
:105040006F008000232E0100EFF08FEA8327C1015B
:10505000138507008320C10213010103678000004C
:10506000130101FE232E110023260100EF00500B37
:1050700097B701009387876F83A70700638A0702AA
:105080009308000013080000930700001307200096
:10509000930600001306004097B50100938585F93B
:1050A000170500001305852EEFC01FEF2326A10072
:1050B0008327C10063960700737004306F000000FF
:1050C0008327C100138507008320C101130101025A
:1050D00067800000130101FC232E1102232EA10082
:1050E000232CB100232AC1002328D1002326E1006C
:1050F0008327810163960700232601026F00800643
:105100001305C002EF10001F2326A1028327C1024E
:10511000638A0704EF00D0008327C1020327C1017F
:1051200023A0E7008327C1020327810123ACE70006
:105130008327C1020327410123AEE7008327C10271
:105140000327010123A0E7028327C1020327C1002F
:1051500023A2E7028327C102938747001385070034
:10516000EFB0CFF48327810163960700737004309A
:105170006F0000008327C102138507008320C1034D
:105180001301010467800000130101FC232E1102AA
:10519000232EA100232CB100232AC1002328D100F3
:1051A0002326E100232601028327C101639607001D
:1051B000737004306F00000097B701009387075B9E
:1051C00083A70700638C070A832781012320F1024C
:1051D000832741012322F1028327C1012324F10205
:1051E000032781019307500063C6E706EFF0CF9DC8
:1051F00013070500930720006318F70297B7010013
:105200009387C75683A70700130701029306000080
:105210000326C1009305070013850700EFB01FD2D6
:105220002326A1026F00800597B7010093870754DA
:1052300083A707001307010293060000130600006E
:105240009305070013850700EFB05FCF2326A10267
:105250006F00C00297B701009387475183A70700EB
:1052600013070102930600000326010193050700BE
:1052700013850700EFB09FF02326A1028327C10208
:10528000138507008320C103130101046780000018
:10529000130101FE2326A1008327C100232EF10064
:1052A0008327C10063960700737004306F0000000D
:1052B0008327C10183A7070013850700130101029B
:1052C00067800000130101FD232611022326A1009F
:1052D0002324B10097B701009387C74883A707002D
:1052E00083A7C70083A7C700232EF1008327C1012E
:1052F0009387470013850700EFB04FF18327C10163
:1053000003A7C701930710006310F7068327C101A5
:1053100003A787018327C100B307F7008326C100D5
:1053200003268100938507000325C101EF00802239
:1053300013070500930710006318F7021307000016
:10534000930600000326C100930500000325C10158
:10535000EFF09FE3232CA1008327810163960700D0
:10536000737004306F0000008327C10183A74702D8
:105370000325C101E7800700130000008320C1025C
:105380001301010367800000130101FD23261102B0
:105390002326A1009307810113850700EF00800EEB
:1053A000232EA10083278101938507000325C101D6
:1053B000EF00C000EF0000286FF0DFFD130101FDDA
:1053C000232611022326A1002324B100EFD01F9829
:1053D0009307810113850700EF004011232EA100E0
:1053E0008327810163960708832781006392070260
:1053F0000327C1008327C10163ECE700EFD05F976B
:105400008325C1010325C100EFF0DFEB6F008006AB
:10541000832781006380070297B701009387C73411
:1054200083A7070083A7070093B7170093F7F70F29
:105430002324F10097B701009387473383A6070021
:105440000327C1008327C101B307F740032681006A
:105450009385070013850600EFC01FABEFD05F9167
:105460009307050063980700EFB08F926F008000EC
:10547000EFD01F90130000008320C102130101032D
:1054800067800000130101FE2326A10097B70100E9
:105490009387472D83A7070083A7070093B71700BB
:1054A00093F7F70F138707008327C10023A0E700B6
:1054B0008327C10083A707006390070297B7010005
:1054C0009387472A83A7070083A7C70083A70700FE
:1054D000232EF1006F008000232E01008327C101DD
:1054E000138507001301010267800000130101FD0D
:1054F000232611022326A100EFD09FA4232EA10072
:1055000097B701009387C72683A707000327C10128
:10551000637CF700EF00C02B8327C1001307100046
:1055200023A0E7006F00C0008327C10023A007006D
:1055300097B701009387C7230327C10123A0E70082
:105540008327C101138507008320C10213010103D2
:1055500067800000130101FD232611022326A1000C
:105560002324B1002322C1002320D100232E0100D7
:105570008327C1000327810023A2E7008327C100FE
:105580000327C10023A8E7000327810083274100E8
:1055900063E6E70403274100832701003307F74050
:1055A0008327C10083A787016368F7009307100072
:1055B000232EF1006F00C00697B701009387C71A2A
:1055C00003A707008327C10093874700938507003F
:1055D00013050700EFB00FB76F00800403274100E9
:1055E00083270100637EF7000327810083270100E2
:1055F0006368F70093071000232EF1006F0040024C
:1056000097B701009387071603A707008327C100F8
:10561000938747009385070013050700EFB08FB20B
:105620008327C101138507008320C10213010103F1
:1056300067800000130101FD232611026F00801511
:105640008327810063C6071483270101232EF100FD
:105650008327C10183A74701638A07008327C1010C
:105660009387470013850700EFB04FBA93074100B7
:1056700013850700EFF09FE7232CA100832781000B
:10568000130790006368F7101397270097B701007E
:105690009387C79AB307F70003A7070097B70100DE
:1056A0009387C799B307F700678007000327C100F6
:1056B0008327C10183A78701B307F7000327C10030
:1056C0009306070003268101938507000325C10186
:1056D000EFF05FE81307050093071000631CF70A5B
:1056E0008327C10183A747020325C101E780070083
:1056F0008327C10103A7C70193071000631CF708A4
:105700000327C1008327C10183A78701B307F700DF
:10571000130700009306000013860700930500009E
:105720000325C101EFF05FA6232AA10083274101D1
:1057300063920706737004306F0000000327C100F6
:105740008327C10123ACE7008327C10183A7870119
:1057500063960700737004306F0000008327C10157
:1057600003A7870183278101B307F70083268101FF
:1057700003268101938507000325C101EFF09FDD1A
:105780006F0040010325C101EF0090566F008000BB
:105790001300000097B70100938747FD83A7070018
:1057A000130781009306000013060000930507000D
:1057B00013850700EFB05FC593070500E39207E884
:1057C000130000008320C102130101036780000061
:1057D000130101FD232611026F00C00E97B70100CF
:1057E000938747F883A7070083A7C70083A707000D
:1057F000232CF10097B701009387C7F683A7070012
:1058000083A7C70083A7C700232AF100832741018C
:105810009387470013850700EFB04F9F832741010F
:1058200083A7470203254101E78007008327410141
:1058300003A7C701930710006316F70883274101E8
:1058400083A7870103278101B307F7002328F1000D
:10585000032701018327810163F0E70483274101C6
:105860000327010123A2E700832741010327410108
:1058700023A8E70097B701009387C7EE03A70700A7
:10588000832741019387470093850700130507008D
:10589000EFB04F8B6F00000313070000930600006A
:1058A000032681019305000003254101EFF0DF8D00
:1058B0002326A1008327C10063960700737004307C
:1058C0006F00000097B701009387C7E983A707001F
:1058D00083A70700E39407F097B70100938787E851
:1058E00083A70700232EF10097B701009387C7E72E
:1058F00003A7070097B701009387C7E623A0E70037
:1059000097B70100938747E60327C10123A0E7006B
:10591000130000008320C10213010103678000000F
:10592000130101FF23261100EFE09FD897B7010074
:105930009387C7E383A707006394070A17B501009D
:105940001305C5DFEFA01FF117B50100130545E0F2
:10595000EFA05FF097B701009387C7E017B701008A
:105960001307C7DD23A0E70097B701009387C7DFC0
:1059700017B701001307C7DD23A0E70013060000D7
:105980009305C00013054000EFB00FA313070500F7
:1059900097B70100938787DD23A0E70097B7010041
:1059A0009387C7DC83A707006396070073700430F2
:1059B0006F00000097B70100938747DB83A70700BC
:1059C0006380070297B70100938747DA83A7070030
:1059D00097A501009385056913850700EFC0CFC225
:1059E000EFE01FD1130000008320C100130101016B
:1059F00067800000130101FD232611022326A10068
:105A00008327C100232EF1008327C100639607007E
:105A1000737004306F000000EFE09FC98327C1015D
:105A200083A74701B337F00093F7F70F232CF1005A
:105A3000EFE01FCC83278101138507008320C1027B
:105A40001301010367800000130101FD23261102E9
:105A50002326A1008327C100232EF1008327C10044
:105A600063960700737004306F000000EFE05FC4BE
:105A70008327C10183A70702232CF100EFE05FC752
:105A800083278101138507008320C10213010103CD
:105A900067800000130101FD232611022326A100C7
:105AA0002324B1008327C100232EF1008327C100E6
:105AB00063960700737004306F000000EFE05FBF73
:105AC0008327C1010327810023A0E702EFE05FC223
:105AD000130000008320C10213010103678000004E
:105AE000130101FE232E11001305C001EF009000E9
:105AF0002326A1008327C100638E07008327C100EE
:105B000023A007008327C100938747001385070060
:105B1000EFA05FD48327C100138507008320C10154
:105B20001301010267800000130101FC232E110202
:105B30002326A1002324B1002322C1002320D10069
:105B40008327C1002324F1022322010203274100FD
:105B5000B70700FFB377F700638607007370043060
:105B60006F000000832741006396070073700430C4
:105B70006F000000EFE05F85930705006396070064
:105B80008327010063960700930710006F008000D1
:105B90009307000063960700737004306F000000E5
:105BA000EFD0CF9A8327810283A707002320F10239
:105BB000832581000325C100EF00804103270102F6
:105BC000832781003367F70083274100B377F7000D
:105BD00003274100631CF70203270102832781008A
:105BE000B367F7002326F1028327810203A707008A
:105BF0008327410093C7F7FF3377F700832781029C
:105C000023A0E700232001006F0040048327010048
:105C10006388070283278102938647000327410098
:105C2000B7070005B367F700032601009385070057
:105C300013850600EFD0DFA4232601026F000001C8
:105C40008327810283A707002326F102EFD04F921A
:105C5000232EA10083270100638407088327C10145
:105C600063940700EFA0DF92EFE05FAE2326A1026E
:105C70000327C102B7070002B377F7006398070450
:105C8000EFE01FA38327810283A707002326F102E9
:105C90000327C10283274100B377F70003274100A0
:105CA0006310F7028327810203A7070083274100BF
:105CB00093C7F7FF3377F7008327810223A0E7001C
:105CC000EFE01FA3930710002322F1020327C10274
:105CD000B70700019387F7FFB377F7002326F10298
:105CE0008327C102138507008320C1031301010428
:105CF00067800000130101FB23261104232EA1005D
:105D0000232CB100232AC1002328D1002326E1003F
:105D10008327C101232AF102232C01022328010237
:105D20008327C10163960700737004306F00000081
:105D300003278101B70700FFB377F70063860700E9
:105D4000737004306F0000008327810163960700A1
:105D5000737004306F000000EFE00FE79307050059
:105D6000639607008327C10063960700930710001E
:105D70006F00800093070000639607007370043083
:105D80006F000000EFC09FFC8327410383A707003B
:105D90002326F10203260101832581010325C10287
:105DA000EF00404B2324A10283278102638C07026A
:105DB0008327C102232EF1022326010083274101FC
:105DC000638807088327410303A70700832781010E
:105DD00093C7F7FF3377F7008327410323A0E7003A
:105DE0006F0000078327C100639807008327C10263
:105DF000232EF1026F00C00583274101638A07004B
:105E000003278103B7070001B367F700232CF102D2
:105E100083270101638A070003278103B707000472
:105E2000B367F700232CF1028327410393864700D1
:105E30000327810183278103B367F7000326C1008D
:105E40009385070013850600EFD09F83232E010260
:105E5000EFC01FF22322A1028327C1006388070835
:105E60008327410263940700EFA08FF2EFE01F8EBB
:105E7000232EA1020327C103B7070002B377F7005F
:105E8000639C0704EFE0DF828327410383A70700B9
:105E9000232EF10203260101832581010325C1037D
:105EA000EF00403B9307050063840702832741010D
:105EB000638007028327410303A70700832781012B
:105EC00093C7F7FF3377F7008327410323A0E70049
:105ED000EFE01F82232801020327C103B707000157
:105EE0009387F7FFB377F700232EF1028327C103CF
:105EF000138507008320C10413010105678000009A
:105F0000130101FD232611022326A1002324B10041
:105F10008327C100232EF1008327C1006396070069
:105F2000737004306F00000003278100B70700FF83
:105F3000B377F70063860700737004306F000000CA
:105F4000EFE00FF78327C10183A70700232CF1009F
:105F50008327C10103A707008327810093C7F7FFA9
:105F60003377F7008327C10123A0E700EFE04FF864
:105F700083278101138507008320C10213010103D8
:105F800067800000130101FD232611022326A100D2
:105F90008327C100232EF100EFA08FFE9307050099
:105FA000232CF1008327C10183A70700232AF100D6
:105FB0008327810113850700EFA0CFFA83274101D2
:105FC000138507008320C1021301010367800000CD
:105FD000130101FB232611042326A1002324B10071
:105FE000232C01028327C1002328F102232A010266
:105FF0008327C10063960700737004306F000000B0
:1060000003278100B70700FFB377F7006386070017
:10601000737004306F0000008327010393874700EB
:106020002326F1028327C102938787002324F102EC
:10603000EFC0DFD18327C10283A7C700232EF1025F
:106040008327010303A70700832781003367F70035
:106050008327010323A0E7006F00000E8327C103FD
:1060600083A747002322F1028327C10383A70700E8
:106070002320F102232A010203270102B70700FFB0
:10608000B377F700232EF10003270102B7070001C1
:106090009387F7FFB377F7002320F1020327C101AD
:1060A000B7070004B377F700639207028327010361
:1060B00003A7070083270102B377F700638807026D
:1060C00093071000232AF1026F0040028327010387
:1060D00003A7070083270102B377F7000327010214
:1060E0006316F70093071000232AF1028327410368
:1060F000638007040327C101B7070001B377F700E6
:10610000638A07000327810383270102B367F7002F
:10611000232CF1028327010303A70700B70700021E
:10612000B367F700938507000325C103EFD05F82B3
:1061300083274102232EF1020327C1038327810213
:10614000E31EF7F08327010303A7070083278103DA
:1061500093C7F7FF3377F7008327010323A0E700F6
:10616000EFC01FC18327010383A707001385070022
:106170008320C1041301010567800000130101FDA4
:10618000232611022326A1008327C100232EF1001C
:106190008327C10193874700232CF100EFC01FBB69
:1061A0006F0040038327810103A7C7008327810174
:1061B000938787006316F700737004306F00000048
:1061C0008327810183A7C700B70500021385070055
:1061D000EFD00FF88327810183A70700E39407FC22
:1061E0000325C101EF00C030EFC09FB813000000CD
:1061F0008320C1021301010367800000130101FE27
:10620000232E11002326A1002324B1008325810021
:106210000325C100EFF0DFDB130000008320C10184
:106220001301010267800000130101FE232E1100FB
:106230002326A1002324B100832581000325C1006A
:10624000EFF01FCC130000008320C10113010102F5
:1062500067800000130101FE2326A1002324B10062
:106260002322C100232E01008327410063900702EF
:106270000327C10083278100B377F70063860702F5
:1062800093071000232EF1006F0000020327C100C6
:1062900083278100B377F700032781006316F70097
:1062A00093071000232EF1008327C10113850700F7
:1062B0001301010267800000130101FE2326A100E3
:1062C0008327C100232CF1008327C10063960700B8
:1062D000232E01006F0000018327810183A787011E
:1062E000232EF1008327C10113850700130101024A
:1062F00067800000130101FC232E11022326A10058
:1063000023220102EFC09FA497370300938787479A
:1063100083A70700639C0700EF00002C973703005A
:10632000938747461307100023A0E7008327C10087
:10633000638A070293078000138707008327C10041
:10634000B387E7002326F1008327C10093F73700C6
:10635000638A07008327C10093F7C7FF938747002D
:106360002326F1008327C100638207160327C1009B
:10637000B79701009387B7FF63EAE71497370300E5
:106380009387473F2324F102973703009387873E83
:1063900083A707002326F1026F0080018327C10233
:1063A0002324F1028327C10283A707002326F102D9
:1063B0008327C10283A747000327C10063F8E700D2
:1063C0008327C10283A70700E39A07FC0327C102C2
:1063D000973703009387873A630AF70E8327810272
:1063E00083A7070013078000B387E7002322F10289
:1063F0008327C10203A707008327810223A0E700A8
:106400008327C10203A747008327C100B307F740D2
:1064100013078000131717006378F7080327C102DA
:106420008327C100B307F700232EF1008327C102A1
:1064300003A747008327C1003307F7408327C10123
:1064400023A2E7008327C1020327C10023A2E7009C
:106450008327C10183A74700232CF100973703004E
:10646000938747312320F1026F0000018327010247
:1064700083A707002320F1028327010283A70700D7
:1064800083A7470003278101E3E2E7FE8327010298
:1064900003A707008327C10123A0E7008327010288
:1064A0000327C10123A0E70097A701009387470FA7
:1064B00003A707008327C10283A747003307F740DC
:1064C00097A701009387C70D23A0E700EFC05F8A5D
:1064D0008327410263940700EF10400D8327410298
:1064E000138507008320C1031301010467800000A6
:1064F000130101FD232611022326A1008327C100D9
:10650000232CF1008327C1006382070A93078000D0
:10651000B307F04003278101B307F700232CF100F4
:1065200083278101232AF100EFC05F828327410185
:1065300083A747002328F100973703009387872319
:10654000232EF1006F0000018327C10183A70700FC
:10655000232EF1008327C10183A7070083A74700EB
:1065600003270101E3E2E7FE8327C10103A7070038
:106570008327410123A0E7008327C10103274101AD
:1065800023A0E7008327410103A7470097A7010045
:106590009387070183A707003307F70097A7010038
:1065A0009387070023A0E700EFC08FFC13000000D3
:1065B0008320C102130101036780000097A7010037
:1065C000938707FE83A707001385070067800000F5
:1065D0001300000067800000130101FF97A701006E
:1065E0009387871993F7C7FF2326F1009737030096
:1065F000938747180327C10023A0E70097370300BC
:106600009387471723A2070097370300938707173D
:10661000379701001307C7FF23A2E700973703004E
:106620009387C71523A007008327C1002324F10007
:1066300083278100379701001307C7FF23A2E700D4
:1066400083278100173703001307471323A0E700B0
:10665000130000001301010167800000130101FE17
:106660002326A1002324B1002322C1008327810017
:10667000232EF1008327C100232CF1000327C10042
:1066800083278100B367F70093F737006396070607
:106690006F00C0028327C10103A707008327810180
:1066A00023A0E7008327810193874700232CF10073
:1066B0008327C10193874700232EF10083274100E0
:1066C0009387D7FF0327C100B307F7000327810192
:1066D000E362F7FC6F0040020327C1019307170034
:1066E000232EF1008327810193861700232CD100EC
:1066F000034707002380E7000327C10083274100E9
:10670000B307F70003278101E368F7FC8327C10083
:10671000138507001301010267800000130101FEC9
:106720002326A1002324B1002322C1000327C10096
:1067300083274100B367F70093F737006398070694
:106740008327810093F7F70F232AF1008327410164
:106750009397870003274101B367F700232AF100CD
:10676000832741019397070103274101B367F7008E
:10677000232AF1008327C100232EF1006F0080013E
:106780008327C10113874700232EE100032741011E
:1067900023A0E7000327C10083274100B307F700C8
:1067A0000327C101E36EF7FC6F00C0038327C1001C
:1067B000232CF1006F00C00183278101138717008C
:1067C000232CE100032781001377F70F2380E700D4
:1067D0000327C10083274100B307F7000327810186
:1067E000E36CF7FC8327C100138507001301010246
:1067F00067800000130101FE2326A1008327C1004A
:10680000232EF1006F0000018327C1019387170039
:10681000232EF1008327C10183C70700E39607FEFB
:106820000327C1018327C100B307F7401385070081
:106830001301010267800000130101FE2326A1005D
:106840002324B1008327C100138717002326E1000A
:1068500083C70700A30FF100832781001387170068
:106860002324E10083C70700230FF1008347F101D0
:10687000638807000347F1018347E101E304F7FC64
:106880000347F1018347E101B307F7401385070090
:106890001301010267800000130101FE2326A100FD
:1068A0002324B1008327C100232EF1001300000030
:1068B00003278100930717002324F1008327C101D8
:1068C00093861700232ED100034707002380E7009B
:1068D00083C70700E39E07FC8327C10013850700D9
:1068E0001301010267800000130101FE2326A100AD
:1068F000232E0100232C01006F0000018327C1001B
:10690000938717002326F1008327C10003C70700E0
:1069100093070002E304F7FE8327C10003C70700C3
:106920009307D002630AF7008327C10003C707005B
:106930009307B0026312F7068327C10083C70700DD
:10694000938737FD93B7170093F7F70F232CF100C8
:106950008327C100938717002326F1006F00C0032F
:106960000327C1019307070093972700B387E70028
:1069700093971700232EF1008327C1001387170078
:106980002326E10083C70700938707FD0327C10182
:10699000B307F700232EF1008327C10083C7070048
:1069A000E39007FC83278101638807008327C101E7
:1069B000B307F0406F0080008327C10113850700F3
:1069C0001301010267800000130101FE2326A100CC
:1069D00097370300938707DF83A707009386170085
:1069E00017370300130707DE2320D7000327C10052
:1069F0001377F70F973603009386C6E0B387F60048
:106A00002380E7000327C1009307A000630CF70071
:106A100097370300938707DB03A70700930700045A
:106A2000631EF704973703009387C7DD232EF10019
:106A30006F00C0038327C10113871700232EE100D5
:106A400003C70700B70710F0938707F023A0E700FC
:106A500097370300938707D783A707001387F7FFAC
:106A600097370300938707D623A0E70097370300E3
:106A7000938747D583A70700E39E07FA9307000093
:106A8000138507001301010267800000130101EB69
:106A90002326111423248114232291142320211549
:106AA000232E3113232C4113232A5113232EA1000B
:106AB000232CB1002328C100232AD1002326E10082
:106AC0002324F10023220101232601128327C10080
:106AD000138A0700930A000083270101032841015C
:106AE00013060A0093860A00138507009305080021
:106AF000EF20C042930705001388050013860700A6
:106B0000930608008327C112138717002326E1127A
:106B1000130706009397270093060113B387F60027
:106B200023AEE7EE8327C10013840700930400001F
:106B3000832741011387040063E8E70483274101A9
:106B4000138704006398E7008327010113070400FB
:106B500063ECE7028327C100138907009309000053
:106B600013060900938609000325010183254101CD
:106B7000EF10105D93070500138805002328F1002E
:106B8000232A01016FF09FF4130000006F00400101
:106B90008327C1018325810103254100E780070088
:106BA000832781001387F7FF2324E1000327C11205
:106BB000E340F7FE6F0040058327C112939727003B
:106BC00013070113B307F70003A7C7EF8327C11209
:106BD0009397270093060113B387F60083A6C7EFA8
:106BE0009307900063F6D700930770056F0080004D
:106BF00093070003B387E7000327C10183258101C1
:106C000013850700E70007008327C1121387F7FFEA
:106C10002326E112E342F0FA130000008320C1149E
:106C20000324811483244114032901148329C113EB
:106C3000032A8113832A4113130101156780000081
:106C4000130101FF2326A1002324B1008326810024
:106C5000130710006356D7028327C10083A70700DC
:106C60009387770093F787FF938687000327C100F8
:106C70002320D70003A8470083A707006F00000563
:106C800003278100630407020327C10003270700CD
:106C9000130647008326C10023A0C6000327070070
:106CA00093070700130800006F0040020327C1008C
:106CB00003270700130647008326C10023A0C60050
:106CC0000327070093070700130800001385070038
:106CD000930508001301010167800000130101FF03
:106CE0002326A1002324B10083268100130710006E
:106CF0006356D7028327C10083A7070093877700D5
:106D000093F787FF938687000327C1002320D700CE
:106D100003A8470083A707006F00800503278100B1
:106D2000630607020327C100032707001306470075
:106D30008326C10023A0C60003270700930707008E
:106D40001357F741130807006F0080020327C100A3
:106D500003270700130647008326C10023A0C600AF
:106D600003270700930707001357F741130807008D
:106D700013850700930508001301010167800000D7
:106D8000130101FC232E1102232C8102232A9102DC
:106D90002326A1002324B1002322C1002320D100F7
:106DA0006F0040026300043C832741009387170073
:106DB0002322F1008327C1008325810013050400ED
:106DC000E78007008327410083C70700138407007B
:106DD00093075002E318F4FC8327410093871700C0
:106DE0002322F100832741002328F10093070002AA
:106DF000A30BF1009307F0FF232EF1009307F0FFA0
:106E0000232CF10023200102832741001387170060
:106E10002322E10083C70700138407009307D4FDF2
:106E2000130750056360F732139727009797010007
:106E300093874724B307F70003A70700979701003C
:106E400093874723B307F700678007009307D002B3
:106E5000A30BF1006FF05FFB93070003A30BF1009E
:106E60006FF09FFA232C010003278101930707008D
:106E700093972700B387E70093971700B307F400B1
:106E8000938707FD232CF1008327410083C7070068
:106E9000138407009307F00263D2870493079003DB
:106EA00063CE870283274100938717002322F100D6
:106EB0006FF09FFB83270100138747002320E10029
:106EC00083A70700232CF1006F0080018327C101F5
:106ED000E3DC07F2232E01006FF01FF31300000024
:106EE0008327C101E3D207F283278101232EF1001A
:106EF0009307F0FF232CF1006FF01FF183270102AD
:106F0000938717002320F1026FF01FF08327010001
:106F1000138747002320E10083A707000327C10050
:106F20008325810013850700E70007006F004023D9
:106F300083270100138747002320E10083A4070073
:106F40006396040097940100938444128327C1013F
:106F50006350F008034771019307D002630AF706F4
:106F6000832781019385070013850400EF10101B10
:106F7000130705008327C101B387E740232EF100E3
:106F80006F004002834771010327C1008325810000
:106F900013850700E70007008327C1019387F7FFE8
:106FA000232EF1008327C101E34EF0FC6F00400265
:106FB0008327C1008325810013050400E7800700B3
:106FC000938414008327C1019387F7FF232EF100D8
:106FD00083C704001384070063000404832781012E
:106FE000E3C807FC832781019387F7FF232CF10077
:106FF00083278101E3DE07FA6F0000028327C100C7
:107000008325810013050002E78007008327C10163
:107010009387F7FF232EF1008327C101E340F0FEA1
:107020006F000014930701008325010213850700F8
:10703000EFF0DFCA93070500138805002324F1024F
:1070400023260103832781020328C1029307080036
:1070500063D607048327C100832581001305D0026E
:10706000E7800700832581020326C1029307000001
:1070700013080000B386B7401385060033B5A70098
:107080003307C840B307A74013870700938706005C
:10709000130807002324F102232601039307A0000D
:1070A0002322F1026F0040069307A0002322F10281
:1070B0006F000004930780002322F1026F00400359
:1070C000930710002320F1028327C100832581004C
:1070D00013050003E78007008327C1008325810093
:1070E00013058007E7800700930700012322F102C0
:1070F000930701008325010213850700EFF05FB4B9
:107100002324A1022326B1020327410283477101F0
:10711000138807008327C101032681028326C10249
:10712000832581000325C100EFF05F966F004003C7
:107130008327C1008325810013050400E780070031
:107140006F0000028327C1008325810013055002D0
:10715000E7800700832701012322F10013000000CC
:107160006FF05FC6130000008320C1030324810376
:10717000832441031301010467800000130101FF10
:107180002326A1006F000000130101FB232611023A
:107190002326A100232AB102232CC102232ED102CF
:1071A0002320E1042322F1042324010523261105D1
:1071B00093070105938747FE232EF1008327C10122
:1071C000938607000326C1009305000017F5FFFF13
:1071D0001305C57FEFF0DFBA9307000013850700A2
:1071E0008320C1021301010567800000130101FE25
:1071F0002326A1002324B1002322710083278100CC
:10720000232EF1008327C10183A707000327C100B4
:107210001377F70F2380E7008327C10183A70700B7
:10722000138717008327C10123A0E7001300000084
:107230001301010267800000130101FA232E1102DD
:107240002326A1002324B1002324C1042326D10432
:107250002328E104232AF104232C0105232E110500
:10726000930701062322F10293074101930541018F
:10727000170600001306C6F737F7FFFF9346F7FF20
:1072800037150000130505803388A5003378E80022
:107290001368783B23A007013305A6003377E50088
:1072A0001367773323A2E70033F7D500931547011F
:1072B000378703001307373933E7E50023A4E700D6
:1072C0003377D60093164701370703001307770675
:1072D00033E7E60023A6E7000F1000008327C10074
:1072E0002326F10293070106938787FE2324F102E8
:1072F0000327810293074101138507009307C1000B
:10730000930607000326810093850700EFF05FA72F
:107310008327C100238007008327C100138707004C
:107320008327C102B307F740138507008320C103F9
:107330001301010667800000130101FE232E1100D6
:107340002326A10017950100130545E8EFF0DFE3C0
:10735000130000008320C1011301010267800000B7
:10736000130101FE232E11002326A1001795010011
:10737000130545E6EFF05FE1130000008320C10133
:107380001301010267800000130101FD2326110291
:107390002326A100232E01006F00400113000000EE
:1073A0008327C10193871700232EF1000327C10112
:1073B000B717000093877738E3D2E7FE17950100EF
:1073C0001305C5E1EFF05FDC6FF0DFFC130101FE98
:1073D000232E1100179501001305C5E0EFF0DFDA49
:1073E0002326010017950100130505E1EFF0DFD911
:1073F000EF00001EEF00D026EF00906C1707000092
:1074000013070708930600001306100093054006B3
:1074100017950100130545DFEFD0DFCB2326A10030
:107420008327C1006388070217950100130585DED5
:10743000EFF09FD5EFB0DFB0930705001307000012
:107440009306000013860700930510000325C10072
:10745000EFD09FD32324010017950100130585DC8D
:10746000EFF09FD2EFB0DF80930700001385070095
:107470008320C1011301010267800000130101FD97
:10748000232611022326A100979701009387071056
:1074900083A7070013874706979701009387070F75
:1074A00023A0E700979701009387470E83A7070063
:1074B00093850700179501001305C5D7EFF0DFCCC2
:1074C000979701009387870C03A70700B717000061
:1074D000938777BB63F4E70C17950100130545D636
:1074E000EFF09FCA232E0100EF00500D1307050097
:1074F00093071000630EF70017950100130505D5DB
:10750000EFF09FC88327C10193E72700232EF100E6
:10751000EF0090501307050093071000630EF7006B
:10752000179501001305C5D4EFF01FC68327C101CD
:1075300093E74700232EF100EF10402D13070500BD
:1075400093071000630EF700179501001305C5D4CB
:10755000EFF09FC38327C10193E78700232EF1003B
:107560008327C101638E0700B7EFEFBE938FDFEA79
:1075700017950100130585D4EFF01FC16F0080013E
:10758000B7CFADDE938FFFEE17950100130505D43D
:10759000EFF09FBFEFB0CFF86F0080001300000046
:1075A0008320C1021301010367800000737004305F
:1075B0006F0000001300000067800000130101FF4E
:1075C0002326A1002324B100737004306F00000053
:1075D000130101FF2326110013060000930540004C
:1075E00013055000EF904FDD1307050097270300A8
:1075F0009387472523A0E7009727030093878724D5
:1076000083A7070097950100938505CD1385070093
:10761000EFA08FFF930800001308000093070000FD
:107620001307200093060000130600409795010001
:107630009385C5CB170500001305C504EFA0DF95A2
:107640009308000013080000972703009387C71FC3
:1076500013071000930600001306004097950100E1
:10766000938545C9170500001305855BEFA0DF92E0
:10767000130000008320C100130101016780000096
:10768000130101FC232E11022326A1002320010255
:107690006F00400B832701021307A000B317F70008
:1076A0002326F102EFB0DF892324A10297270300EC
:1076B0009387471983A707001307C10193060000AA
:1076C0000326C1029305070013850700EF90DFD35F
:1076D00093070500638A070097270300938787179E
:1076E0001307100023A0E700EFB09F8513070500E4
:1076F00083278102B307F7402322F10203274102C7
:107700008327C102637AF7009727030093878714C2
:107710001307100023A0E7008327C1029387F70017
:107720000327410263FAE700972703009387871234
:107730001307100023A0E700832701029387170097
:107740002320F1020327010293074000E3D4E7F46A
:10775000232001026F000005972703009387870EFF
:1077600083A7070013070102930600001306000019
:107770009305070013850700EF904FFC13070500E2
:1077800093071000630AF700972703009387870C7D
:107790001307100023A0E700832701029387170037
:1077A0002320F1020327010293074000E3D6E7FA02
:1077B000232001026F00400B832701021307A00062
:1077C000B317F7002326F102EFB08FF72324A102AD
:1077D000972703009387070783A707001307010272
:1077E000930600000326C1029305070013850700D6
:1077F000EF90CFF493070500638A070097270300F3
:10780000938747051307100023A0E700EFB04FF35D
:107810001307050083278102B307F7402322F102F3
:10782000032741028327C102637AF70097270300E9
:10783000938747021307100023A0E7008327C102A4
:107840009387F7000327410263FAE70097270300B5
:10785000938747001307100023A0E7008327010246
:10786000938717002320F1020327010293074000AA
:10787000E3D4E7F497270300938707FE23A00700CC
:1078800097270300938747FC83A70700138507000A
:10789000EFB04F9B6F00C00013054001EFA0DFBBAE
:1078A00097270300938747FB03A70700930750051B
:1078B000E314F7FE13054001EFA01FBA972703005A
:1078C000938787F923A00700232001026F0080100F
:1078D00097270300938707F783A707001307C101C2
:1078E00093060000130600009305070013850700A8
:1078F000EF909FB11307050093071000630AF7008C
:1079000097270300938707F51307100023A0E700CC
:1079100097270300938707F383A707001307010244
:107920009306000013060000930507001385070067
:10793000EF90CFE01307050093071000630AF700EC
:1079400097270300938707F11307100023A0E70090
:1079500097270300938747F003A707009307500575
:10796000631AF700972703009387C7EE13071000E9
:1079700023A0E70097270300938707ED83A707005D
:107980009305400013850700EFA0DFD09727030081
:10799000938787EC03A7070093075005631AF70046
:1079A00097270300938707EB1307100023A0E70036
:1079B00097270300938747E983A7070093051000E3
:1079C00013850700EFA01FCD8327010293871700BF
:1079D0002320F1020327010293074000E3DAE7EED8
:1079E0006F00C00013054001EFA01FA797270300F9
:1079F000938787E603A7070093075005E314F7FE74
:107A000013054001EFA05FA5972703009387C7E404
:107A100023A00700232001026F0000059727030021
:107A2000938747E283A707001307C101930600006D
:107A3000130600009305070013850700EF90DF9CF5
:107A40001307050093071000630AF7009727030048
:107A5000938747E01307100023A0E7008327010264
:107A6000938717002320F1020327010293074000A8
:107A7000E3D6E7FA97270300938707DD83A707007C
:107A800013850700EFA01FFC6F00C0001305400125
:107A9000EFA09F9C97270300938707DC03A70700AD
:107AA00093075005E314F7FE13054001EFA0DF9A9A
:107AB00097270300938747DA23A0070023200102BA
:107AC0006F008010972703009387C7D783A707000D
:107AD0001307010293060000130600009305070038
:107AE00013850700EF908FC513070500930710005B
:107AF000630AF700972703009387C7D51307100081
:107B000023A0E700972703009387C7D383A7070025
:107B10001307C10193060000130600009305070038
:107B200013850700EF905F8E130705009307100081
:107B3000630AF700972703009387C7D11307100044
:107B400023A0E70097270300938707D103A7070027
:107B500093075005631AF70097270300938787CF91
:107B60001307100023A0E700972703009387C7CDD2
:107B700083A707009305400013850700EFA09FB17E
:107B800097270300938747CD03A707009307500566
:107B9000631AF700972703009387C7CB13071000DA
:107BA00023A0E70097270300938707CA83A707004E
:107BB0009305100013850700EFA0DFAD83270102B6
:107BC000938717002320F102032701029307400047
:107BD000E3DAE7EE6F00C00013054001EFA0DF8796
:107BE00097270300938747C703A70700930750050C
:107BF000E314F7FE13054001EFA01F86972703004B
:107C00009387C7C483A7070013871700972703002C
:107C10009387C7C323A0E7006FF05FA7130101FD9F
:107C2000232611022326A10013050000EFA0DFC6C2
:107C3000EFB00FB1232EA100232A010097270300E4
:107C4000938787C11307500523A0E70097270300F8
:107C5000938747BF83A707001307410193060000DE
:107C60001306F00A9305070013850700EF900FAD88
:107C700093070500638A070097270300938787BD52
:107C80001307100023A0E700EFB08FAB1307050028
:107C90008327C101B307F740232CF100032781019B
:107CA0009307E00A63EAE70097270300938787BA00
:107CB0001307100023A0E700032781019307E00BBF
:107CC00063FAE700972703009387C7B813071000EC
:107CD00023A0E70097270300938707B813075005F1
:107CE00023A0E70013050000EFA01FBBEFB04FA5D6
:107CF000232EA10097270300938707B6130750058B
:107D000023A0E700972703009387C7B383A7070043
:107D100013074101930600001306F00A93050700BC
:107D200013850700EF904FEE93070500638A070065
:107D300097270300938707B21307100023A0E700DB
:107D4000EFB00FA0130705008327C101B307F74069
:107D5000232CF100032781019307E00A63EAE7007F
:107D600097270300938707AF1307100023A0E700AE
:107D7000032781019307E00B63FAE70097270300CD
:107D8000938747AD1307100023A0E7009727030050
:107D9000938787AC1307500523A0E70097270300BC
:107DA000938707AB83A70700138717009727030064
:107DB000938707AA23A0E7006FF01FE7130101FFD5
:107DC000930710002326F10097270300938707A845
:107DD00003A7070097270300938747A883A70700F7
:107DE0006314F7002326010097270300938747A613
:107DF00003A7070097270300938787A683A7070099
:107E00006314F7002326010097270300938787A4B4
:107E100003A70700930710006314F700232601004F
:107E2000972703009387C7A203A70700972703009C
:107E3000938707A323A0E70097270300938707A151
:107E400003A7070097270300938747A123A0E70014
:107E50008327C1001385070013010101678000001B
:107E6000130101FF232611009305800C1305800CDC
:107E7000EF90CF8413070500972703009387C79ED1
:107E800023A0E700972703009387079E1307A00A04
:107E900023A2E700972703009387079D23A40700E9
:107EA000930500001305800CEF904F811307050028
:107EB000972703009387479B23A6E7009727030094
:107EC0009387879A23A80700972703009387C7996A
:107ED00023AA0700972703009387079983A7070022
:107EE000978501009385854113850700EF90DFF1A9
:107EF000972703009387479783A7C70097850100BB
:107F00009385C54013850700EF901FF09727030066
:107F10009387879583A70700639A07009727030035
:107F20009387879483A7C70063820706930800009E
:107F300013080000930700001307000097260300B2
:107F40009386869213060040978501009385053D30
:107F50001705000013054521EFA00F8493080000CA
:107F60001308000093070000130700009726030082
:107F70009386469013060040978501009385853AC5
:107F8000170500001305451EEFA00F811300000028
:107F90008320C1001301010167800000130101FD6E
:107FA000232611022326A1002324B10093060000FA
:107FB00013060000930500000325C100EF801FF8A1
:107FC0001307050093071000631AF70097270300B3
:107FD000938747891307100023A0E700232E010091
:107FE0006F00400593060000130600009305000093
:107FF0000325C100EF904FC1130705009307100040
:10800000630AF700972703009387C78513071000BB
:1080100023A0E7008327810083A7070013871700A9
:108020008327810023A0E7008327C10193871700DE
:10803000232EF1000327C1019307700CE3F4E7FA44
:108040009306000013060000930500000325C100FD
:10805000EF908FBB1307050093071000631AF7001A
:1080600097270300938707801307100023A0E700DA
:10807000130000008320C102130101036780000088
:10808000130101FD232611022326A1002324B100A0
:108090009306000013060000930500000325C100AD
:1080A000EF908FB61307050093071000631AF700CF
:1080B000971703009387077B1307100023A0E7009F
:1080C000232E01006F0040059306000013060000F8
:1080D000930500000325C100EF805FE6130705004C
:1080E00093071000630AF7009717030093878777B9
:1080F0001307100023A0E7008327810083A7070050
:10810000138717008327810023A0E7008327C1017D
:1081100093871700232EF1000327C1019307700CEA
:10812000E3F4E7FA9306000013060000930500004D
:108130000325C100EF809FE013070500930710009F
:10814000631AF700971703009387C771130710008E
:1081500023A0E700130000008320C10213010103E4
:1081600067800000130101FD232611022326A100D0
:108170008327C100232EF1008327C10103A74700F5
:108180009307A00A6310F7028327C10103A7070022
:108190008327C10193878700938507001305070094
:1081A000EFF0DFDF8327C10183A7070093060000FC
:1081B000130600009305000013850700EF90CFA47D
:1081C0001307050093071000631AF70097170300C1
:1081D000938747691307100023A0E7008327C10195
:1081E00003A707008327C1019387870093850700B2
:1081F00013050700EFF0DFE88327C10103A707009D
:108200008327C10193878700938507001305070023
:10821000EFF0DFD86FF09FFC130101FF9307100010
:108220002326F100971703009387C76383A70700EE
:108230006384070023260100971703009387C76212
:1082400003A78700971703009387876383A7070017
:108250006316F700232601006F00C0019717030083
:108260009387876003A78700971703009387476169
:1082700023A0E700971703009387075F03A7470131
:10828000971703009387076083A707006316F7001B
:10829000232601006F00C001971703009387C75C76
:1082A00003A74701971703009387C75D23A0E70043
:1082B0008327C100138507001301010167800000B7
:1082C000130101FF2326110013054000EF80DF9DFD
:1082D00013070500971703009387075B23A0E700A8
:1082E000971703009387475A83A7070097850100D4
:1082F0009385C50313850700EF901FB197170300FF
:108300009387875883A707006388070893080000AE
:1083100013080000971703009387C758130720001E
:108320009306000013060040978501009385050120
:108330001705000013058507EF901FC6930800007E
:1083400013080000971703009387075613071000C0
:10835000930600001306004097850100938585FE73
:10836000170500001305C51AEF901FC393080000FE
:108370001308000093070000130700009306000095
:108380001306004097850100938545FC1705000002
:1083900013050529EF905FC0130000008320C10082
:1083A0001301010167800000130101FD2326110262
:1083B0002326A100971703009387074D83A7070083
:1083C00013850700EF801F9B13070500930710001C
:1083D000631AF700971703009387474B13071000A2
:1083E00023A0E700232E01006F00C00497170300AD
:1083F0009387874983A707009305800013850700AB
:10840000EF80DFA01307050093071000630AF70051
:1084100097170300938787471307100023A0E700EF
:1084200013054001EFA04F838327C10193871700F5
:10843000232EF1000327C10193079000E3F8E7FA28
:10844000232E01006F00800413054001EFA0CF80B0
:10845000971703009387474383A7070013850700F7
:10846000EF805F911307050093071000630AF70080
:1084700097170300938787411307100023A0E70095
:108480008327C10193871700232EF1000327C10121
:1084900093079000E3FAE7FA971703009387C73E24
:1084A00083A7070013850700EF80DF8C1307050003
:1084B00093071000631AF700971703009387073D8F
:1084C0001307100023A0E700971703009387C73C0A
:1084D00083A7070013871700971703009387C73BED
:1084E00023A0E700971703009387873A130710002C
:1084F00023A0E70013050000EFA00FBA97170300B1
:108500009387073923A007006FF0DFEA130101FE0C
:10851000232E11002326A100971703009387C73647
:1085200083A707009305E0FF13850700EF801F8EE8
:1085300013070500930710006312F708971703004D
:108540009387073503A7070093071000630CF70014
:1085500097170300938787331307100023A0E700C2
:108560006F00C006971703009387073283A70700A1
:1085700013850700EF801F80130705009307100085
:10858000630AF7009717030093874730130710001B
:1085900023A0E700971703009387C72F1307100046
:1085A00023A0E70013050000EFA00FAF971703000B
:1085B0009387472E23A007006F0040019717030001
:1085C0009387C72C1307100023A0E7009717030019
:1085D0009387C72C83A707001387170097170300FB
:1085E0009387872B83A70700630AF7009717030079
:1085F0009387C7291307100023A0E70097170300EC
:108600009387C72983A707001387170097170300CD
:108610009387C72823A0E7006FF01FF0130101FE26
:10862000232E11002326A100971703009387C72547
:1086300083A707009305000013850700EF800FFD57
:108640001307050093071000E310F7FE97170300C8
:108650009387472583A7070013850700EF90DFE87E
:1086600013070500930730006306F70073700430AA
:108670006F000000971703009387072383A7070065
:1086800013850700EF905FE613070500930730009E
:108690006306F700737004306F0000009717030043
:1086A0009387471F03A7070093071000631CF70079
:1086B000971703009387C71D03A7070093071000B0
:1086C000630CF700971703009387471C13071000EC
:1086D00023A0E7006F004013971703009387471C00
:1086E00083A7070013871700971703009387471B7B
:1086F00023A0E700971703009387071B83A70700B2
:1087000013850700EFA00FB497170300938787190D
:1087100083A7070013850700EFA0CFB297170300C8
:108720009387471703A7070093071000630CF70010
:10873000971703009387C71503A707009307100037
:10874000631AF70097170300938747141307100065
:1087500023A0E70013050000EF905FE81307050072
:10876000930720006306F700737004306F00000069
:10877000971703009387071383A707001385070044
:10878000EF909FD613070500930720006306F700BC
:10879000737004306F000000971703009387C710B1
:1087A00083A7070013850700EF901FD41307050068
:1087B000930720006306F700737004306F00000019
:1087C000971703009387470C83A7070013850700BB
:1087D000EF804FDA1307050093071000630AF700D4
:1087E000971703009387870A1307100023A0E70059
:1087F00013050000EF909FDE93070500E38607E274
:10880000737004306F0000006FF01FE2130101FF6E
:10881000971703009387870903A70700971703009B
:108820009387870783A70700631CF7009717030048
:108830009387C7051307100023A0E7006F00C0014E
:10884000971703009387470503A7070097170300AF
:108850009387C70523A0E700971703009387470571
:1088600003A70700971703009387470383A7070011
:10887000631CF70097170300938747011307100045
:1088800023A0E7006F00C00197170300938707013B
:1088900003A70700971703009387870123A0E7002A
:1088A000971703009387070103A707009717030093
:1088B000938707FF83A70700631CF7009717030040
:1088C0009387C7FC1307100023A0E7006F00C001C7
:1088D000971703009387C7FC03A7070097170300A8
:1088E000938747FD23A0E70097170300938707FAB4
:1088F00003A70700930710006316F7002326010063
:108900006F00C000930710002326F1008327C100E9
:10891000138507001301010167800000B305B5004E
:10892000930705006386B70003C7070063160700B7
:108930003385A74067800000938717006FF09FFE84
:10894000130101FD23286101232671012326110251
:10895000232481022322910223202103232E31018B
:10896000232C4101232A5101232481012322910137
:108970002320A101130B0500938B0500639E06388D
:108980003709028093040600130A0500130909350C
:1089900063F8C512B7070100138405006378F61069
:1089A0001307F00F3337C70013173700B357E6002C
:1089B0003309F900834609003387E6009306000275
:1089C000B386E640638C06003394DB003357EB003C
:1089D000B314D60033648700331ADB0093DA040142
:1089E00093850A0013050400EF00902A93090500FF
:1089F00093850A0013050400139B0401EF00D024A3
:108A0000135B0B01130905009305050013050B000B
:108A1000EF00D0209399090193570A01B3E7F900B9
:108A20001304090063FEA700B38797001304F9FF3E
:108A300063E8970063F6A7001304E9FFB387970084
:108A40003389A74093850A0013050900EF005024DD
:108A50009309050093850A0013050900EF00D01E55
:108A6000131A0A01130905009305050093990901DA
:108A700013050B00135A0A01EF00501A33EA49019B
:108A800013060900637CAA00338A44011306F9FF28
:108A900063669A006374AA001306E9FF13140401C5
:108AA0003364C400930A00006F000013B70700018D
:108AB00013070001E36CF6EE130780016FF01FEF60
:108AC00093890600631A0600930500001305100041
:108AD000EF00901793040500B707010063FEF4123E
:108AE0009307F00F63F4970093098000B3D7340124
:108AF0003309F900034709009306000233073701E1
:108B0000B386E6406394061233849B40930A1000B8
:108B100013DB040193050B0013050400EF0050174D
:108B20009309050093050B0013050400939B0401B2
:108B3000EF00901193DB0B0113090500930505006D
:108B400013850B00EF00900D9399090193570A01CB
:108B5000B3E7F9001304090063FEA700B387970089
:108B60001304F9FF63E8970063F6A7001304E9FF15
:108B7000B38797003389A74093050B0013050900BD
:108B8000EF0010119309050093050B001305090070
:108B9000EF00900B131A0A01130905009305050055
:108BA0009399090113850B00135A0A01EF0010076E
:108BB00033EA490113060900637CAA00338A4401A1
:108BC0001306F9FF63669A006374AA001306E9FFAF
:108BD000131404013364C4001305040093850A00D0
:108BE0008320C1020324810283244102032901025C
:108BF0008329C101032A8101832A4101032B010139
:108C0000832BC100032C8100832C4100032D010024
:108C10001301010367800000B707000193090001F9
:108C2000E3E6F4EC930980016FF05FECB394D400B9
:108C3000B3D9EB0013D404013357EB00B39BDB0033
:108C40009305040013850900B36B7701331ADB0029
:108C5000EF001004130905009305040013850900B3
:108C6000139B0401EF00407E135B0B019309050089
:108C70009305050013050B00EF00407A1319090155
:108C800013D70B013367E900938A0900637EA700BD
:108C900033079700938AF9FF636897006376A7000C
:108CA000938AE9FF33079700B309A74093050400AF
:108CB00013850900EF00C07D93050400130905002A
:108CC00013850900EF0040781304050093050500A3
:108CD00013050B00EF00807413970B011357070166
:108CE00013190901B367E9001307040063FEA70025
:108CF000B38797001307F4FF63E8970063F6A700B4
:108D00001307E4FFB3879700939A0A013384A740BF
:108D1000B3EAEA006FF0DFDF63ECD51EB7070100AE
:108D200063F4F6041307F00FB335D70093953500BD
:108D30003707028013070735B3D7B600B387E700BC
:108D400003C70700930A00023307B700B38AEA405B
:108D500063960A0213041000E3E076E93336CB0091
:108D6000134416006FF05FE7B70700019305000199
:108D7000E3E0F6FC930580016FF09FFBB35CE60037
:108D8000B3965601B3ECDC00B3D4EB00B3975B01B0
:108D900093DB0C013357EB0093850B001385040024
:108DA0003364F700B3195601EF00806E1309050014
:108DB00093850B0013850400139C0C01EF00C06821
:108DC000135C0C01930405009305050013050C00CA
:108DD000EF00C06413190901135704013367E90058
:108DE000138A0400637EA70033079701138AF4FFF8
:108DF000636897016376A700138AE4FF330797013E
:108E0000B304A74093850B0013850400EF0040686E
:108E10001309050093850B0013850400EF00C06261
:108E2000930405009305050013050C00EF00005F97
:108E3000931704011319090193D70701B367F900C8
:108E40001386040063FEA700B38797011386F4FF1F
:108E500063E8970163F6A7001386E4FFB3879701E1
:108E600013140A01B70B01003364C4001389FBFF1C
:108E7000337D240133F92901B384A7409305090008
:108E800013050D00EF008059935C04019305090060
:108E9000130A050013850C00EF00405893D909010F
:108EA000130C05009385090013850C00EF00005793
:108EB000130905009385090013050D00EF00005606
:108EC0003305850193570A013385A7006374850133
:108ED0003309790193570501B387270163E6F4024B
:108EE000E392F4BCB70701009387F7FF3375F500F1
:108EF00013150501337AFA0033165B01330545017A
:108F0000930A0000E37AA6CC1304F4FF6FF09FB934
:108F1000930A0000130400006FF01FCC130101FB43
:108F20002324810423229104232E3103232291033D
:108F30002326110423202105232C4103232A510336
:108F40002328610323267103232481032320A10303
:108F5000232EB101930C050093890500130405002D
:108F600093840500639E0626B70A02801309060053
:108F7000138A0600938A0A3563F4C514B707010003
:108F80006376F6129307F00F63F4C700130A8000AC
:108F9000B3574601B38AFA0003C70A00130500025B
:108FA00033074701330AE540630C0A00B3954901D2
:108FB00033D7EC0033194601B364B70033944C0146
:108FC000935A090193850A0013850400EF00404C71
:108FD0009309050093850A00131B090113850400FA
:108FE000EF008046135B0B019305050013050B0092
:108FF000EF00C0429399090193570401B3E7F900C8
:1090000063FAA700B387270163E6270163F4A7008B
:10901000B3872701B384A74093850A001385040012
:10902000EF0000479309050093850A0013850400AB
:10903000EF00804113140401930505009399090181
:1090400013050B0013540401EF00403D33E4890085
:10905000637AA40033042401636624016374A400CA
:10906000330424013304A440335544019305000024
:109070008320C104032481048324410403290104BF
:109080008329C103032A8103832A4103032B01039C
:10909000832BC102032C8102832C4102032D010288
:1090A000832DC1011301010567800000B70700018E
:1090B000130A0001E36EF6EC130A80016FF05FED16
:1090C000631A06009305000013051000EF00C03777
:1090D00013090500B7070100637AF90E9307F00F33
:1090E00063F42701130A8000B3574901B38AFA00D9
:1090F00003C70A0013050002B3842941330747015F
:10910000330AE540E30E0AEA33194901B3DAE9000C
:10911000B395490133D7EC0093540901336BB70081
:1091200013850A0093850400EF008036930905003B
:1091300093850400931B090113850A00EF00C030DA
:1091400093DB0B019305050013850B00EF00002D49
:109150009399090193570B01B3E7F90033944C013C
:1091600063FAA700B387270163E6270163F4A7002A
:10917000B3872701B38AA7409385040013850A00AB
:10918000EF000031930905009385040013850A0060
:10919000EF00802B9305050013850B00EF000028DE
:1091A00093150B019399090193D50501B3E5B90016
:1091B00063FAA500B385250163E6250163F4A500E4
:1091C000B3852501B384A5406FF09FDFB707000189
:1091D000130A0001E36AF9F0130A80016FF0DFF06F
:1091E000E3E8D5E8B707010063FCF604930BF00F42
:1091F00033B5DB001315350037070280B3D7A6005F
:1092000013070735B387E70083CB070093050002F8
:10921000B38BAB00338B7541631E0B0263E43601E5
:1092200063EACC003384CC40B386D94033B58C009C
:10923000B384A64013050400938504006FF05FE338
:10924000B707000113050001E3E8F6FA13058001F2
:109250006FF09FFAB3966601335D7601336DDD00E2
:1092600033D47901B395690133DC7C0193540D014A
:10927000336CBC001305040093850400B31A660127
:10928000EF000021130A0500938504001305040074
:1092900033996C01931C0D01EF00001B93DC0C0152
:1092A000130405009305050013850C00EF0000175B
:1092B000131A0A0113570C013367EA00130A04005A
:1092C000637EA7003307A701130AF4FF6368A701B1
:1092D0006376A700130AE4FF3307A701B309A74089
:1092E0009385040013850900EF00801A938504001C
:1092F0001304050013850900EF0000159305050010
:109300009304050013850C00EF00401193150C0128
:109310001314040193D50501B365B4001387040049
:1093200063FEA500B385A5011387F4FF63E8A501DB
:1093300063F6A5001387E4FFB385A501131A0A019C
:10934000B70C0100336AEA001384FCFFB3778A008C
:1093500033F48A00B384A540138507009305040005
:109360002326F100135A0A01EF00400B9309050070
:109370009305040013050A00EF00400A13DC0A01FC
:10938000930D050093050C0013050A00EF0000097A
:109390008327C100130A050093050C0013850700FD
:1093A000EF00C0073305B50113D709013307A70044
:1093B0006374B701330A9A01B70701009387F7FF77
:1093C000935507013377F70013170701B3F7F90037
:1093D000B3854501B307F70063E6B400639EB400AC
:1093E000637CF90033865741B3B7C700B385A54105
:1093F000B385F54093070600B307F9403339F90008
:10940000B385B440B385254133947501B3D7670163
:109410003365F400B3D565016FF09FC513060500F1
:109420001305000093F61500638406003305C5009C
:1094300093D5150013161600E39605FE678000000D
:109440006340050663C605061386050093050500FF
:109450001305F0FF630C060293061000637AB60052
:109460006358C0001316160093961600E36AB6FE02
:109470001305000063E6C500B385C5403365D5001C
:1094800093D6160013561600E39606FE678000007A
:1094900093820000EFF05FFB1385050067800200F8
:1094A0003305A04063D80500B305B0406FF0DFF985
:1094B000B305B04093820000EFF01FF93305A040E0
:1094C000678002009382000063CA0500634C0500B8
:1094D000EFF09FF71385050067800200B305B040E9
:1094E000E35805FE3305A040EFF01FF63305B0400A
:0494F000678002008F
:02000004800278
:1000000049444C45000000007C4BFEFF144BFEFFB2
:10001000304BFEFF484BFEFF584BFEFF4C4DFEFFA2
:10002000E44CFEFF004DFEFF184DFEFF284DFEFF85
:10003000546D7220537663007456FEFF7456FEFFB3
:100040007456FEFF5C57FEFF0457FEFF4C57FEFF41
:100050007456FEFF7456FEFF5C57FEFF0457FEFF0A
:10006000546D725100000000286E756C6C29000000
:10007000986DFEFFD470FEFFC070FEFFD470FEFFCF
:10008000D470FEFFD470FEFFD470FEFF446EFEFFFE
:10009000D470FEFFD470FEFFDC6DFEFF5C6EFEFFD1
:1000A000D470FEFFE86DFEFFF46DFEFFF46DFEFF01
:1000B000F46DFEFFF46DFEFFF46DFEFFF46DFEFFC8
:1000C000F46DFEFFF46DFEFFF46DFEFFD470FEFFD5
:1000D000D470FEFFD470FEFFD470FEFFD470FEFF1C
:1000E000D470FEFFD470FEFFD470FEFFD470FEFF0C
:1000F000D470FEFFD470FEFFD470FEFFD470FEFFFC
:10010000D470FEFFD470FEFFD470FEFFD470FEFFEB
:10011000D470FEFFD470FEFFD470FEFFD470FEFFDB
:10012000D470FEFFD470FEFFD470FEFFD470FEFFCB
:10013000D470FEFFD470FEFFD470FEFFD470FEFFBB
:10014000D470FEFFD470FEFFD470FEFFD470FEFFAB
:10015000D470FEFFD470FEFFD470FEFFD470FEFF9B
:10016000D470FEFFD470FEFFD470FEFFD470FEFF8B
:100170009C6EFEFFB46FFEFFD470FEFFD470FEFFD6
:10018000D470FEFFD470FEFFD470FEFFD470FEFF6B
:10019000D470FEFF8C6EFEFFD470FEFFD470FEFFA5
:1001A0004470FEFF5070FEFFD470FEFFD470FEFF5F
:1001B000C06EFEFFD470FEFF3870FEFFD470FEFFED
:1001C000D470FEFF7870FEFF6D69616F750A0000E4
:1001D0006D69616F75320A0068756E6772790A0021
:1001E0006672656552544F532064656D6F20626F6F
:1001F0006F740A00437265617465207461736B7378
:100200000A000000436865636B54696D6572000005
:1002100053746172742074696D65720A0000000085
:100220005374617274206B65726E656C0A00000015
:100230007469636B2025640D0A00000063686563C0
:100240006B20210D0A0000004572726F7220696EEA
:1002500020626C6F636B2074696D652074657374C4
:10026000207461736B73200D0A0000004572726F79
:100270007220696E20636F756E74696E6720736596
:100280006D6170686F7265207461736B73200D0A05
:10029000000000004572726F7220696E2072656303
:1002A000757273697665206D7574657820746173F5
:1002B0006B73200D0A0000004572726F7220666F2A
:1002C000756E6421200D0A005041535321200D0A00
:1002D00000000000426C6F636B5F54696D655F5195
:1002E0007565756500000000425465737431000047
:1002F0004254657374320000436F756E74696E67A3
:100300005F53656D5F310000436F756E74696E6792
:100310005F53656D5F320000434E543100000000B2
:10032000434E543200000000526563757273697663
:10033000655F4D757465780052656331000000009B
:100340005265633200000000526563330000000014
:10035000000102020303030304040404040404046C
:10036000050505050505050505050505050505053D
:10037000060606060606060606060606060606061D
:10038000060606060606060606060606060606060D
:1003900007070707070707070707070707070707ED
:1003A00007070707070707070707070707070707DD
:1003B00007070707070707070707070707070707CD
:1003C00007070707070707070707070707070707BD
:1003D000080808080808080808080808080808089D
:1003E000080808080808080808080808080808088D
:1003F000080808080808080808080808080808087D
:10040000080808080808080808080808080808086C
:10041000080808080808080808080808080808085C
:10042000080808080808080808080808080808084C
:10043000080808080808080808080808080808083C
:10044000080808080808080808080808080808082C
:100450001000000000000000037A5200017C01013E
:100460001B0C02008800000018000000D484FEFF6E
:10047000DC0500000004040000000E300430000021
:1004800000960897098101880289039204930594D4
:10049000069507980A990B9A0C04700200000AC18D
:1004A0000404000000C80404000000C904040000A3
:1004B00000D20404000000D30404000000D40404AB
:1004C000000000D50404000000D60404000000D79A
:1004D0000404000000D80404000000D90404000053
:1004E00000DA04040000000E0004040000000B0009
:1004F00090000000A4000000248AFEFF0005000018
:100500000004040000000E5004340000008802893A
:10051000039305990B810192049406950796089719
:1005200009980A9A0C9B0D04200100000AC10404DA
:10053000000000C80404000000C90404000000D248
:100540000404000000D30404000000D404040000EC
:1005500000D50404000000D60404000000D7040401
:10056000000000D80404000000D90404000000DAF0
:100570000404000000DB04040000000E000404007A
:0405800000000B006C
:10058C00AAAAAAAA40FF0FF048FF0FF0080000002B
:08059C00FC8F010004000000C7
:040000058000004037
:00000001FF
